:020000040007F3
:1020000080930020D9230700E1230700E323070082
:10201000E5230700E7230700E9230700000000008D
:10202000000000000000000000000000C5230700C1
:10203000ED23070000000000EF230700F123070055
:10204000F3230700F3230700F3230700F32307001C
:10205000F3230700F3230700F3230700F32307000C
:10206000F3230700F3230700F3230700F3230700FC
:10207000F3230700F3230700F3230700F3230700EC
:10208000F1360700F3230700F3230700F3230700CB
:10209000F3230700F323070061350700F32307004C
:1020A000F3230700F3230700F3230700F3230700BC
:1020B000F3230700F32307000000000000000000E6
:1020C000F3230700F3230700F3230700F32307009C
:1020D0005D340700F3230700F3230700F323070011
:1020E000F3230700000000000000000000000000D3
:1020F00000000000F323070000000000F3230700A6
:1021000000000000000000000000000000000000CF
:1021100000000000000000000000000000000000BF
:1021200000000000000000000000000000000000AF
:10213000000000000000000000000000000000009F
:10214000000000000000000000000000000000008F
:10215000000000000000000000000000000000007F
:10216000000000000000000000000000000000006F
:10217000000000000000000000000000000000005F
:10218000000000000000000000000000000000004F
:10219000000000000000000000000000000000003F
:1021A000000000000000000000000000000000002F
:1021B000000000000000000000000000000000001F
:1021C000000000000000000000000000000000000F
:1021D00000000000000000000000000000000000FF
:1021E00000000000000000000000000000000000EF
:1021F00000000000000000000000000000000000DF
:10220000DFF810D000F050F900480047415A0700AD
:10221000AFF300808093002030B450E8012F93B2D8
:10222000C48923448489A34228BF1B1B0489A34279
:1022300002BFBFF32F8F002007E0C3EA020340E88C
:102240000134002CE9D14FF001000A6030BC704726
:1022500050E8012FC2EA024240E801210029F7D1EB
:10226000704730B450E8022F1FFAA2F3C488A3428B
:1022700002BFBFF32F8F00200DE0C489234484895F
:10228000A34228BF1B1BC2EA034340E80234002CD0
:10229000E8D14FF001000A6030BC704750E8022FCF
:1022A000C2EA224240E802210029F7D170470346E2
:1022B00053E8022FD988B2EB324F4FF0000017BF1E
:1022C00092B241EA014142EA014104E05A68B2EBAC
:1022D000324F08BF012043E80212002AE8D17047BC
:1022E00030B4044654E8000F0D4644E80053002B78
:1022F000F8D1156030BC704730B4044654E8000F84
:1023000040EA010544E80053002BF7D1156030BCCA
:10231000704730B4044654E8000F00EA010544E871
:102320000053002BF7D1156030BC704730B4044621
:1023300054E8000F80EA010544E80053002BF7D170
:10234000156030BC704730B4044654E8000F00EB11
:10235000010544E80053002BF7D1156030BC7047ED
:1023600030B4044654E8000FA0EB010544E80053E4
:10237000002BF7D1156030BC704770B404464FF0A5
:10238000000054E8006F0D68AE4207BF44E8002328
:10239000012044E800630E60002B1CBF0020F0E722
:1023A00070BC704730B4044654E8000F88422CBF1C
:1023B000451A054644E80053002BF5D1156030BCA2
:1023C000704700001EF0040F0CBFEFF30880EFF31E
:1023D000098007F06FBA00000648804706480047AA
:1023E000FEE7FEE7FEE7FEE7FEE7FEE7FEE7FEE7C5
:1023F000FEE7FEE76535070001220700202A04DB1F
:10240000203A00FA02F1002070479140C2F1200307
:1024100020FA03F3194390407047000000487047CA
:1024200000CB070040EA01039B0703D009E008C97D
:10243000121F08C0042AFAD203E011F8013B00F889
:10244000013B521EF9D27047D2B201E000F8012BD5
:10245000491EFBD270470022F6E710B513460A4624
:1024600004461946FFF7F0FF204610BD421C10F845
:10247000011B0029FBD1801A704730B504460020AB
:10248000034600E05B1C934203D2E05CCD5C401B42
:10249000F8D030BD034611F8012B00F8012B002ABB
:1024A000F9D1184670470000064C074D06E0E06879
:1024B00040F0010394E8070098471034AC42F6D38B
:1024C000FFF7A2FE00DB070020DB07002DE9F04349
:1024D0008BB01446129D15F9046B00961F4680467A
:1024E00089462B460246214602A800F086FC02A936
:1024F000129A084600F07DFC129B02AA4146404613
:1025000000F067FC129B02AA2146204600F061FC05
:102510002B464A4639463846009600F06EFC129A21
:10252000394602A800F065FC02A92B46424608463F
:10253000009600F062FC02A92B462246084600964F
:1025400000F05BFC2B46424621462046009600F0F8
:1025500054FC129B22464946484600F03AFC2B4662
:1025600002AA41462046009600F047FC129B2246F4
:102570003946384600F02DFC2B464A463946384647
:10258000009600F03AFC324602A9204600F0FCFD1D
:102590000BB0BDE8F083F0B5154689B01C46074680
:1025A0000E461A462946684600F023FC23466A4632
:1025B0003946384600F00DFC23462A4669466846EF
:1025C00000F007FC23466A463146304600F001FC25
:1025D00009B0F0BD8B1802448B4200D1704713F84C
:1025E000010D02F8010DF7E72DE9F047B3F90240BC
:1025F00088461E4604F11F012023073491FBF3F7A0
:1026000008234FFA87F994FBF3F4944228BF144649
:102610004946054600F072FA22464146FFF7DAFFC6
:10262000B6F90230E4009C421FD9E41A05EB870199
:102630000022C4F120078D420ED324364A46294693
:10264000304600F066FA01280FD04B463246284645
:10265000BDE8F04700F0A4BD51F8040D20FA04F3E2
:1026600013430B6000FA07F2E5E7BDE8F0872DE9B8
:10267000F04793F9006092B004468946104631460F
:102680001546984600F05AFA002840F091804246DC
:10269000494602A800F0ADFB434602AA21460AA81B
:1026A00000F097FB02A90846424600F0A2FB434611
:1026B0002A464946484600F08CFB08F1040742468A
:1026C0002946284600F095FB3B462A4621462046EF
:1026D000009600F042FA3B462A46294628460096D4
:1026E00000F03BFA3B462A4621462846009600F079
:1026F00084FB43462A462146204600F06AFB3B46BF
:10270000224621462846009600F027FA3B460096CE
:102710002A462146204600F020FA2368DB074AD5E6
:1027200033463A462146204600F0BAF93146824601
:10273000204600F01CFD06F18043013B54F82300C5
:1027400040EACA7044F8230042462146284600F079
:1027500050FB3B460AAA29462846009600F04DFB4E
:102760003B460AAA29462846009600F046FB0AA9DD
:1027700008463B462A46009600F03FFB43460AAA1D
:102780002146204600F025FB02AA3B461046214682
:10279000009600F032FB32462946204600F0F4FC59
:1027A0004946284600F0F0FC02A9484600F0ECFC3F
:1027B00012B0BDE8F0873146204600F0D8FCC3E7F0
:1027C0000048704750DA07002DE9F04FEDB01F4682
:1027D000DDF8D8810590B8F9026098F9004020230F
:1027E0001F3696FBF3F676B206F1FF3924AB0025CF
:1027F00043F829506CAB03EB89034CA88A469346F7
:10280000394698F9012043F8805C43F8605CFFF793
:10281000E1FE98F9012054A8B918FFF7DBFE214624
:102820004CA800F08BF90746002840F02E8154A8F0
:1028300000F084F90290002840F0298108F1240377
:1028400032464CA91846039300F063F9012840F082
:102850002081324654A9039800F05BF901280690C4
:1028600040F017811CAD0CAF3346039A54A928469B
:1028700000F08CF9029B47F829305A4651463846F9
:102880004346FFF7B1FE39463846039B00962A4679
:1028900000F0FFF90DF5B879039B00962A464CA984
:1028A00014A800F0F6F922464846059900F06CFCA1
:1028B000A30009EB030A0793059BA100591808F12F
:1028C000440B504600F060FC594634A800F05CFC14
:1028D000A3000BEB03013CA800F056FC08F1040335
:1028E000494634AA28460094049300F086FA5346D9
:1028F0004A463CA934A8CDF80080FFF7E7FD2346FF
:10290000049A2946284600F041F92A46514648468D
:102910004346FFF740FE029BCDE9083B059B31464D
:102920003846CDE90A3900F003FC3146814614A847
:1029300000F0FEFB8145B8BF81461FFA89F909F115
:10294000FF3B0FFA8BFB5946384600F059FC5946BD
:10295000071C14A818BF012700F052FC002814BF60
:10296000022300231F430DF1200A22465AF8277044
:1029700024A8394600F008FC0DF1B00BA300F918AB
:10298000584600F001FC2146284600F0B7F8A9F1AE
:102990000209069B2B600FFA89F90DF1900AB9F133
:1029A000000F23DA2346049A2946284600F0EEF861
:1029B00043462A4659465046FFF7EDFD32465146FA
:1029C000039800F0A6F8012804D03346039A504635
:1029D00000F0E6FB013C64B24CAA23064BD5029BF7
:1029E000B3FA83F040096DB0BDE8F08F43462A4644
:1029F000D8F8A47059465046B84749460CA800F08C
:102A0000FFFB4946071C14A818BF012700F0F8FB7C
:102A1000002814BF022300231F4308AB53F827707C
:102A200027B32246394634A800F0AEFB079B3CA8EA
:102A3000F91800F0A9FB43462A463CA934A8FFF741
:102A4000AAFD049B009434AA514644A800F0D5F98D
:102A50005B4652463CA934A8CDF80080FFF736FD0E
:102A6000434644AA2946284600F0B3F909F1FF3944
:102A70000FFA89F993E752F824105AF824304B40A2
:102A8000029919430291013CA7E72846ABE7384673
:102A9000A9E70298A7E7000000000000000000007E
:102AA000C3F10803DB0070B50133002403A500BFA8
:102AB0005B1920C940CAAD1920C0184720C940CAB7
:102AC000754120C020C940CA754120C020C940CAF4
:102AD000754120C020C940CA754120C020C940CAE4
:102AE000754120C020C940CA754120C020C940CAD4
:102AF000754120C06441204670BD00BF002310B561
:102B00001C465AB2914200DC10BD40F8234001330C
:102B1000F7E710B5013A52B2130601D5002010BDF7
:102B200050F8224051F822309C4205D802F1FF3281
:102B3000F2D24FF0FF30F2E70120F0E710B50023AA
:102B40001A465CB2A14203DCB2FA82F0400910BD21
:102B500050F8234001332243F3E770B59DF910404C
:102B60001E4623460546FFF79BFF30B922462946FD
:102B70003046FFF7CEFF012807D0234632462946CC
:102B80002846BDE8704000F00BBB70BDF0B50F46A5
:102B9000A1B006461946384615461C46FFF7CEFF3B
:102BA00020B13046FFF7AAFF21B0F0BD22463946DA
:102BB000684600F0E9FA294608A800F0E5FA10A8EE
:102BC0002146FFF79BFF012318A81093FFF796FFFC
:102BD000224608A96846FFF79CFF28B9224610A99B
:102BE000304600F0D1FADFE7009BDA0709D421462E
:102BF000684600F0BCFA2246294610A800F0E0FB27
:102C0000E6E7089BDB0707D4214608A800F0AFFAE7
:102C10002246294618A8F1E7002823461CDD08AA09
:102C20006946684600F0BCFA2146684600F09FFA03
:102C3000224618A910A8FFF76CFF002805DA10A992
:102C400023462A460846FFF72BFF10A9234618AA59
:102C5000084600F0A5FACEE708A96A46084600F043
:102C60009FFA214608A800F082FA224610A918A867
:102C7000FFF74FFF002805DA18A923462A46084621
:102C8000FFF70EFF18A9234610AA084600F088FA9D
:102C9000BEE72DE9F04FB5B004AD9DF9F8401F46F1
:102CA00081462346284600F0BAF824AB2146384630
:102CB000CDE9023500F03CFAC0EB841005B26B425E
:102CC00003F01F034FF0200695FBF6F676B205F0F1
:102CD0001F0814A858BFC3F100083146FFF70EFFC4
:102CE000B8F1000F30B22DDD14AB002203EB8000F1
:102CF000C8F1200C1346A34219D327B27B000193DD
:102D000014AB03EB870704F1FF3834AB012603EB68
:102D10008808002D53DA34AB03EB8606224656F8BA
:102D2000C81C484600F030FA35B0BDE8F08F57F8BF
:102D3000236006FA08F10A4340F8232026FA0CF231
:102D40000133D8E714AB2246394603EB800000F08C
:102D50001BFAD2E70FFA82FE5AF8C83C53F82EB09D
:102D600034AB03EB820252F8803CABEB03031B1A3B
:102D70009B4502D034BF012000205CF8C82C42F8EB
:102D80002E300131019B4AB29A42E3DB331A5E4294
:102D9000214614A85E4100F0EAF934AB03EB84034A
:102DA000214653F8802C58F8803C384643EAC273D9
:102DB000013D48F8803C2DB200F0D9F9A9E734ABC9
:102DC0000021C6F1010C084603EB860A03EB8C0CCC
:102DD000D8E730B51C4691B0054693F900306846F7
:102DE00000F01DF8D4F8AC3069462846984711B079
:102DF00030BD13460A46FFF7ECBF70B59DF9104091
:102E00001E462346054600F0CBF938B1234632462C
:102E100029462846BDE87040FFF742BE70BD2DE947
:102E2000F04F08B4F8CA04B451F8042BA3FB02898C
:102E300040F8048B4FF0000AE4FB629A4FF0000B5D
:102E4000E5FB62AB4FF0000CE6FB62BC4FF0000EFE
:102E5000E7FB62CE51F8042B4FF00008E3FB6289D8
:102E600040F8048BE4FB629AE5FB62ABE6FB62BCD4
:102E7000E7FB62CE51F8042B4FF00008E3FB6289B8
:102E800040F8048BE4FB629AE5FB62ABE6FB62BCB4
:102E9000E7FB62CE51F8042B4FF00008E3FB628998
:102EA00040F8048BE4FB629AE5FB62ABE6FB62BC94
:102EB000E7FB62CE51F8042B4FF00008E3FB628978
:102EC00040F8048BE4FB629AE5FB62ABE6FB62BC74
:102ED000E7FB62CE40F8049B40F804AB40F804BB2B
:102EE00040F804CB40F804EB0CBC052B00F01E812D
:102EF0000C68A0F11400A1F11401A2F1140252F81F
:102F000004EB4FF0000550F8046BE4FB6E5652F8EA
:102F100004EB50F8047BE4FB6E6752F804EB50F8C6
:102F2000048BE4FB6E7852F804EB50F8049BE4FB4E
:102F30006E8952F804EB50F804ABE4FB6E9AA0F1F2
:102F4000140052F8044B51F804EB4FF0000CE4FB72
:102F50006EC540F804CB51F804EBE4FB6E5640F824
:102F6000045B51F804EBE4FB6E6740F8046B51F826
:102F700004EBE4FB6E7840F8047B51F804EBE4FBCF
:102F80006E8940F8048B51F804EBE4FB6E9AA0E8DC
:102F90000006062B00F0CA800C68A0F11800A1F111
:102FA0001801A2F1180252F804EB4FF0000550F896
:102FB000046BE4FB6E5652F804EB50F8047BE4FB20
:102FC0006E6752F804EB50F8048BE4FB6E7852F80D
:102FD00004EB50F8049BE4FB6E8952F804EB50F8C4
:102FE00004ABE4FB6E9A52F804EB50F804BBE4FB2C
:102FF0006EABA0F1180052F8044B51F804EB4FF0FF
:10300000000CE4FB6EC540F804CB51F804EBE4FB84
:103010006E5640F8045B51F804EBE4FB6E6740F831
:10302000046B51F804EBE4FB6E7840F8047B51F834
:1030300004EBE4FB6E8940F8048B51F804EBE4FBED
:103040006E9A40F8049B51F804EBE4FB6EABA0E8E9
:10305000000C072B6AD008B40C68A0F11C00A1F189
:103060001C01A2F11C0252F804EB4FF0000550F8CD
:10307000046BE4FB6E5652F804EB50F8047BE4FB5F
:103080006E6752F804EB50F8048BE4FB6E7852F84C
:1030900004EB50F8049BE4FB6E8952F804EB50F803
:1030A00004ABE4FB6E9A52F804EB50F804BBE4FB6B
:1030B0006EAB52F804EB50F804CBE4FB6EBCA0F10D
:1030C0001C0052F8044B51F804EB4FF00003E4FBF2
:1030D0006E3540F8043B51F804EBE4FB6E5640F8C3
:1030E000045B51F804EBE4FB6E6740F8046B51F8A5
:1030F00004EBE4FB6E7840F8047B51F804EBE4FB4E
:103100006E8940F8048B51F804EBE4FB6E9A40F8AA
:10311000049B51F804EBE4FB6EAB40F804AB51F8B0
:1031200004EBE4FB6EBCA0E8001808BCBDE8F08F1F
:10313000013949B20A06CBB205D4013900EB81024C
:103140005268002AF6D001335BB273B103F18042BA
:10315000013A50F82220002022B9013B00EB431332
:1031600018B2704752080130F6E71846704700EB76
:1031700081010023884200D3704751F8042D43EAAF
:1031800052030B60D307F5E710B500235CB2A242EF
:1031900000DC10BD51F8234040F823400133F5E72F
:1031A000C3F10803DB0070B50133002403A500BFA1
:1031B0005B1920C940CAAD1B20C0184720C940CAAE
:1031C000B54120C020C940CAB54120C020C940CA6D
:1031D000B54120C020C940CAB54120C020C940CA5D
:1031E000B54120C020C940CAB54120C020C940CA4D
:1031F000B54120C06441B4FA84F0400970BD00BFFD
:103200004A11012350F8220001F01F0103FA01F1D5
:1032100008407047F0B5082289B00C460646FFF713
:10322000B3FFCB6A03930B6B04934B6B05938B6BD0
:103230000693CB6B0793002708236A4669466846C6
:10324000CDE901770097FFF72BFC082305466A4676
:1032500031463046FFF724FC236B0393636B0493E2
:10326000A36B0593E36B0544CDE906376A46082353
:1032700069466846FFF714FC082305446A46314650
:103280003046FFF70DFC236A0093636A0193A36A3B
:103290000293A36B0693E36B0793054408236A46E6
:1032A00031463046CDE904770397FFF7F9FB636AAF
:1032B0000093A36AA26B0193E36A02930492636B87
:1032C000E26B0393CDE90523236A079305440823A2
:1032D0006A4631463046FFF7E3FBE36A0093236B0F
:1032E0000193636B0293236A0693A36A07930544D1
:1032F00008236A4631463046CDE904770397FFF745
:103300004FFF236B0093636B0193A36B0293E36BFB
:103310000393636A0693E36A07932D1A08236A46A8
:1033200031463046CDE90477FFF73AFF636B0093EF
:10333000A36B0193E36B0293236A0393636A049381
:10334000A36ACDE90537236B07932D1A08236A4634
:1033500031463046FFF724FFA36B0093E36BCDE9C2
:103360000137636A0393A36A0493E36ACDE90537DF
:10337000636B07932D1A08236A4631463046FFF7E0
:103380000FFF2D1A0D4C0FD435B9082231462046B7
:10339000FFF7BFFB01280FD00823224631463046F5
:1033A000FFF7FEFE2D1AEFE708232246314630468E
:1033B000FFF776FB2D18F7D409B0F0BD54DA0700FB
:1033C00070B5036813F001050646144605D0134690
:1033D0000A460146FFF764FB054621463046FFF7E3
:1033E000C6FE45B104F18042013A56F8223043F05E
:1033F000004346F8223070BD2DE9F0438BB00446FF
:10340000154689460AAE1C22002103A8FFF725F8BD
:10341000032346F8203D95F900802A464946204678
:103420002F1DFFF7E6FC3B46324621462046CDF8ED
:103430000080FFF7E2FC2B464A4621462046FFF774
:10344000C8FCCDF800803B4605F1840221462046A9
:10345000FFF783FB0BB0BDE8F08300002DE9F041DE
:103460001E4E4FF48271D6F8040130B11C48C26878
:10347000521CC260304605F041FF00254FF4A07792
:1034800007EB85018AB23046B25812B389B205F013
:1034900035FF1348103000EB0514204608F076FD88
:1034A000104811492246401AC008042101EB00408F
:1034B0000EA105F0E5FC616819B1204608F0BCFCDE
:1034C00007E0A16811B1204608F0B6FC206800B101
:1034D00080476D1C022DD3D3BDE8F081004002402F
:1034E000F42A002088DB070038DB070074696D656B
:1034F000725F66697265202830782578290000009F
:1035000000F006B970B50E46144900EB400001EB1F
:10351000C0051446E86A183520B101280FD00228EA
:1035200005D113E0284600F029F9A04201D2002479
:1035300011E022463146284600F058F90BE02846B3
:1035400000F01CF9A042F4D20446F2E731462846C6
:1035500000F01FF90446204670BD0000F86200200C
:1035600006F0A6B810B54FF080520023D2E94C10F7
:103570000D2906D18C07C4F80C31C4F81031534C16
:1035800023600D2955D1524B1B68524C2360504B80
:103590001B1D1B68241D23604D4B08331B68241D15
:1035A00023604B4B0C331B68241D2360484B1033A6
:1035B0001B68241D2360464B14331B68241D2360A5
:1035C000434B18331B68434C20342360404B1C335F
:1035D0001B68241D23603E4B20331B68241D236081
:1035E0003B4B24331B68241D2360394B28331B6855
:1035F000241D2360364B2C331B68241D2360344B61
:1036000030331B68334C40342360314B34331B68F8
:10361000241D23602E4B38331B68241D23602C4B44
:103620003C331B68241D2360294B40331B68241D39
:1036300023600D2906D128480168C90702D06FF020
:10364000010101602548016841F470010160BFF388
:103650004F8FBFF36F8FD2E94C104FF010220D291E
:1036600007D130B1012804D0D2F80802174920311F
:103670000860D2F80002002803DBD2F80402002818
:103680001FDA012006F064F91221C2F80012144872
:103690000368002BFCD0C2F8041201680029FCD09A
:1036A000002006F055F9BFF34F8F0C487C380168B5
:1036B0000C4A01F4E06111430160BFF34F8F00BF7A
:1036C000FDE70A490848086010BD000038050040C1
:1036D0000404001020C500400004004088ED00E014
:1036E00000E401400400FA050090D003F02B002014
:1036F000064808B5002101600068009005F074FCE0
:1037000005F04AFA0028FBD108BD00000001014085
:1037100010B5124C02202061606111A0A06104F17B
:103720007800E0614FF4805020620020A062606267
:103730000BA1A164E0620D49E1641021A065C4E918
:103740001410E0650AA1E01DFEF7A4FE09A12046C1
:10375000FEF7A0FE2020A07110BD0000F86200203E
:103760005465726D696E616C00000000707300201A
:103770005254540053454747455200000269C168FE
:103780008A4203D88068401A104400E0501A401E54
:1037900070472DE9F047C4681746894606464FF042
:1037A00000083069A04201D9051B02E0B168201A67
:1037B0000D1AB0686D1E001BA84200D80546BD4218
:1037C00000D33D4670682A4620444946FEF72AFE4B
:1037D000B0687F1B2C44A844A944A04200D1002417
:1037E000F460002FDDD14046BDE8F0872DE9F041BF
:1037F00004468846D4E90207C51BE168606816469E
:103800000844B54206D94146FEF70CFEB819E060FF
:10381000BDE8F0812A464146FEF704FE761B08EB20
:10382000050132466068FEF7FDFDE660F0E702E064
:1038300008C8121F08C1002AFAD17047704700203B
:1038400001E001C1121F002AFBD17047012120288D
:1038500003DA81400548014003E0402802DA2038BD
:10386000814009B10120704700207047FC06FFBD70
:10387000800701D000207047012070474068006831
:10388000401E084201D10120704700207047C368E4
:103890008B4206D811440069491E814201D801209B
:1038A000704700207047000030B585B00D46164CBB
:1038B0001621ADF800101ECC0DF1040C8CE81E0092
:1038C000124C0221012221706270A0700320E0706E
:1038D000217159206071FE20A071694604F1090030
:1038E0007DDF00280ED1BDF800002A46411CE171A1
:1038F00009212172BDF808100844ADF8080001A99B
:10390000034872DF05B030BDC0C507002830002075
:103910002C2B002010B586B0062418220D496846CD
:10392000FEF780FD0C480D49401AC008042101EB48
:1039300000400BA105F0A0FA69462046FFF7B4FF4E
:10394000002805D10A4C207874DF0121207873DF2C
:1039500006B010BDD0C5070040DB070038DB07000C
:103960004164766572746973696E672E2E2E00004D
:103970002C2B00202DE9F05FDFF89CB05C46DBF8D3
:103980004890DBF8246003F00BF8216B4718751A98
:1039900022482349401AC108042000EB0140804618
:1039A00020A105F069FA216B4944B94200D10025F4
:1039B00008232A46384601F0D1FD07001848174968
:1039C0004FF0010AA1EB00004FEAD0010AEB0144DD
:1039D00004D020461AA105F04FFA19E002F0E0FFEA
:1039E0000022314601F0E6F9DBF828200546D946E9
:1039F000AA4208D1404619A105F03EFAC9E9075A82
:103A0000C9F8186004E020462B461A4905F03FFA31
:103A10003846BDE8F09F0000C047002088DB070063
:103A200038DB0700456E746572206E72665F6466EF
:103A3000755F6170705F636F6E74696E75650000AD
:103A40004661696C656420746F20636F70792066CD
:103A500069726D776172652E0000000053657474A1
:103A6000696E67206170702061732076616C696493
:103A700000000000F0CB070008B513460246009393
:103A80000648074BC01AC008012303EB00400B4651
:103A900004A105F004FA06F0F5FB000088DB07003E
:103AA00038DB0700526563656976656420612066CE
:103AB00061756C74212069643A203078253038783B
:103AC0002C2070633A203078253038782C20696EAD
:103AD000666F3A2030782530387800000246064874
:103AE0000649401AC008012101EB004004A105F07D
:103AF000C7F906F0C7FB000088DB070038DB0700CA
:103B0000526563656976656420616E206572726FC7
:103B1000723A203078253038782100002DE9F041C4
:103B200007461E4E1E481F49326A401AC508012A20
:103B300004D0032000EB05401BA12BE04FF44050C4
:103B4000184B174C4168E31A234A0220DB0800EBAC
:103B50000344914206D1C1023B462048726B00F0FB
:103B60004FFF90B102F01CFF01461C483B4641301C
:103B7000B26900F045FF58B1042000EB054018A1E0
:103B800005F07AF90120BDE8F081204618A101E096
:103B9000204626A105F070F90020F4E7C047002078
:103BA00088DB070038DB0700426F6F742076616C9A
:103BB00069646174696F6E206661696C65642E204A
:103BC0004E6F2076616C69642061707020746F2084
:103BD000626F6F742E000000DBE5B151204A0020B7
:103BE0004170702069732076616C69640000000088
:103BF000426F6F742076616C69646174696F6E20C6
:103C00006661696C65642E20536F667444657669DD
:103C100063652069732070726573656E74206275C8
:103C20007420696E76616C69642E0000426F6F7457
:103C30002076616C69646174696F6E206661696C7D
:103C400065642E2041707020697320696E76616C06
:103C500069642E002DE9F84F254C81469246608814
:103C60000E46814241D800274FF6FF788DF800704C
:103C7000684600F075F822786078A188884201DAF9
:103C8000401C00E00020C0B2904204D19DF800002A
:103C900000F0B2F827E065786078884201DA401CCD
:103CA00000E0002060709DF8000000F0A5F8454598
:103CB00019D0A068B9F1000F40F835A00DD066B159
:103CC0006188E068324605FB01004946FEF7AAFB21
:103CD000A06800EBC500868002E000EBC50087808D
:103CE0000020BDE8F88F0420FBE70920F9E7000079
:103CF000702B002010B50E4C03E0401C00E00020AB
:103D0000207020786178814210D022786188E06844
:103D1000A36802FB010003EBC20153F8322089883B
:103D200090472078A1888842E9DAE6E710BD0000D4
:103D3000702B002030B5CB0008339DB293074FF0B5
:103D4000000401D0072030BD044B9A602A44DA6099
:103D50005C701C7058809980002030BD702B002052
:103D600070B5044607F056F9012803D010A143208E
:103D700000F086F8EFF3108172B61D4A93680120B7
:103D800083B990604FF0E020D0F88051194B1D406E
:103D90001560C0F88031D0F8843153604217C0F804
:103DA000842100202070002900D162B670BD00007F
:103DB0002E2E5C2E2E5C2E2E5C2E2E5C2E2E5C6308
:103DC0006F6D706F6E656E74735C6C696272617238
:103DD0006965735C7574696C5C6170705F7574693A
:103DE0006C5F706C6174666F726D2E630000000012
:103DF000344F0020FC06FFBD10B5044607F00AF959
:103E0000012803D00DA1512000F03AF81B49886821
:103E1000002811D0002C0FD1EFF3108072B60B6880
:103E20004FF0E022C2F800314B68C2F804310022A2
:103E30008A60002800D162B610BD00002E2E5C2ED4
:103E40002E5C2E2E5C2E2E5C2E2E5C636F6D706FA2
:103E50006E656E74735C6C69627261726965735CC5
:103E60007574696C5C6170705F7574696C5F706C9F
:103E70006174666F726D2E6300000000344F002085
:103E80001CB56A46CDE90001002144F20200FFF7AB
:103E9000F3FD1CBDF8B521480146456AC06A8C6C2B
:103EA000AC2801D024B106E0486B04442D1A02E08E
:103EB00002F08AFD04461A481A492346401AC708E8
:103EC000042000EB07400646174A18A1009504F0AD
:103ED000E6FF2A4621461448FEF7CFFAD0B1304615
:103EE0002B4622461FA104F0D2FF00BF04F054FE6F
:103EF0000028FBD102F028FB2946204603F04CF9AC
:103F0000040005D0012000EB074022A104F0B4FF1B
:103F10002046F8BD0024304625A1F7E7C047002021
:103F200088DB070038DB0700002007005665726950
:103F30006679696E6720424C3A20416464723A2087
:103F40003078253038782C205372633A2030782529
:103F50003038782C204C656E3A203078253038780F
:103F600000000000436F7079696E6720626F6F74A4
:103F70006C6F616465723A205372633A2030782521
:103F80003038782C204C656E3A20307825303878DF
:103F9000000000005265717565737420746F2063B2
:103FA0006F707920424C206661696C656400000086
:103FB0004E6F20626F6F746C6F6164657220636F07
:103FC0007079206E65656465642C20626F6F746C17
:103FD0006F616465722075706461746520636F6DD4
:103FE000706C6574652E000030B595B0040004D186
:103FF0002E4940F24F40FFF743FF2D494FF6FF7027
:104000002246488001208DF812004FF65960ADF825
:10401000100004A90120A8DF002844D1254B0FCBB4
:104020008DE80F00A11C684662DF00283BD12149C2
:104030001C2260390BA8FEF7F5F91F4D142205F17B
:10404000C401A8681290A0788DF84A0028681390DF
:1040500006A8FEF7E7F912A8069013A80790208893
:10406000231D06AA0BA9AADF00281CD11C2205F1DA
:10407000D8010BA8FEF7D6F9E8681290A0788DF861
:104080004A0068681390142205F1F40106A8FEF7AF
:10409000C9F912A8069013A80790208804F10C0310
:1040A00006AA0BA9AADF15B030BD0000DCCC0700C2
:1040B0002C2B002098C6070090C50700F0B585B0EE
:1040C0000D46040004D1374940F28710FFF7D8FEAF
:1040D00025B934494FF4C470FFF7D2FE1421684665
:1040E000FEF7B9F92078032308280BD12E48C188A0
:1040F000491E89B2C1808288002A4BD0002949D14B
:10410000C28023702178607860228DF800208DF8BD
:1041100001108DF8020063780325012B16D0234887
:1041200023492278401AC008022101EB004021A156
:1041300004F0ADFE60780B2828D101F04FF98DF81E
:104140000300002001F052F904251FE0207809281F
:104150001CD2DFE800F01B1B1B211B1B051B2100D1
:10416000D4E902706D46E91C666807F035FF044625
:1041700029193046C91C07F02FFF04442919384675
:10418000C91C07F029FF2044C01CC5B22946684657
:1041900007F008F805B0F0BDD4E90112684606F052
:1041A000F0FFF1E7DCCC07002C2B002040DB070000
:1041B00038DB0700444655207265717565737420BD
:1041C0002564206661696C65642077697468206580
:1041D00072726F723A203078257800002DE9F04134
:1041E0001D4C0026217AC90733D01C49884230D0A3
:1041F0001B481C49401AC108042000EB0140054639
:1042000019A104F039FE6088A0F57F41FF3916D06E
:1042100028461DA104F030FEA068132140F00400E0
:10422000A060608876DF002814D11B4CC8264FF4AC
:104230007A47611C38468847761EFAD101E020781B
:1042400074DF05F0D1F9060003D1284613A104F06C
:1042500013FE3046BDE8F0812C2B002020DB070048
:1042600040DB070038DB07005368757474696E67BC
:1042700020646F776E20424C45207472616E7370BB
:104280006F72742E00000000446973636F6E6E6578
:104290006374696E672E0000A0C50700424C45207C
:1042A0007472616E73706F727420736875742064B9
:1042B0006F776E2E0000000070B5204C064600207F
:1042C000217AC90738D11E481E49401AC108042066
:1042D00000EB014005461CA104F0CEFD2248E6603B
:1042E00001F0B4FD00F01CFB002825D103F02AF9F1
:1042F00038B11E4803F01AF9A06840F00200A0602F
:1043000003E028461AA104F0B7FD01F0BBF800282D
:1043100012D116481C30FFF767FE00280CD1FFF7BA
:10432000F9FA002808D1A06818A140F00100A060A7
:10433000284604F0A1FD002070BD00002C2B0020B9
:1043400040DB070038DB0700496E697469616C69FE
:104350007A696E6720424C4520444655207472614C
:104360006E73706F72740000A8DB07004830002085
:104370004E6F206164766572746973696E67206E32
:10438000616D6520666F756E64000000424C4520CB
:10439000444655207472616E73706F727420696E3A
:1043A000697469616C697A65642E00002DE9FE43C9
:1043B0009F49A04B0122591AC9080746051D02EB67
:1043C0000148008804229C4E4FF0000902EB014492
:1043D00021286ED037DC13286CD01EDC01286AD06F
:1043E000102854D0112868D0122879D1204693A1E2
:1043F00004F042FDEA8820469AA104F041FDAA8813
:1044000020469EA104F03CFD2A892046A1A104F08B
:1044100037FD6A892046A4A1ECE0142875D01A283B
:1044200074D01F285CD12046A5A104F025FD291DCC
:10443000708875DF040053D040462246ACA104F0DA
:104440001FFD20461FE051287AD00EDC222878D0AC
:10445000232868D024287BD0502877D103B0394650
:10446000BDE8F043B04805F09DBF5228D8D055288C
:1044700037D056286AD1B879002867D113217088BF
:1044800076DF002862D0BDE8FE43FFF727BB204659
:10449000A6A104F0F1FC28887080F16809B1012020
:1044A0008847A549708875DF02004FD04046A3A118
:1044B000A0E07FE055E087E0FFE74FF6FF707080F7
:1044C000307A400704D4FFF725FA08B1FFF706FB5E
:1044D000F16800293AD003B00220BDE8F043084754
:1044E00034E0FA88F72A14D29007B0F1404F0ED08A
:1044F000D01F81B2481EC31700EB937323F0030350
:10450000C01A081A801D85B204E078E081E01546E3
:1045100000E0F72520462B46944904F0B8FC2946D4
:104520007088B5DFADE7204691A104F0A5FCCDF879
:104530000090CDF80490B8880022694690DF2DE005
:1045400046E02EE004E000BFFFF7C8FABDE8FE83B6
:104550006B89EA8803B02046BDE8F04391A104F0DE
:1045600096BC20469FA104F087FC734801AA163828
:1045700042F60521806A0190CDF808D07088ADDF41
:1045800008B1FFF7ABFA2046BDF800209FA104F068
:1045900077FC00231A46852170887FDF0028D3D15D
:1045A000D4E7287900906B79AA792046A0A104F07D
:1045B00076FCCBE72046ADA104F05EFCCDF8009080
:1045C000288869468FDFE9E70021708866DF58E7B1
:1045D000B8790028BAD03946534805F09FFE002824
:1045E000B4D007F10801504805F0B8FA0200ADD088
:1045F0004046A9A103B0BDE8F04304F041BC204609
:10460000B2A104F039FC00210A4628880B4686DF57
:1046100037E7002328881A461946B1DF08B1FFF7AB
:104620005DFA03B02046BDE8F043B2A104F024BC1B
:1046300038DB070040DB07002C2B00205265636548
:104640006976656420424C455F4741505F4556544A
:104650005F434F4E4E5F504152414D5F5550444174
:10466000544500006D61785F636F6E6E5F696E74B4
:10467000657276616C3A2025640000006D696E5F9A
:10468000636F6E6E5F696E74657276616C3A202539
:1046900064000000736C6176655F6C6174656E63C5
:1046A000793A202564000000636F6E6E5F73757049
:1046B0005F74696D656F75743A20256400000000B1
:1046C000526563656976656420424C455F47415099
:1046D0005F4556545F434F4E4E5F504152414D5FD0
:1046E0005550444154455F5245515545535400007F
:1046F0004661696C75726520746F207570646174B1
:104700006520636F6E6E656374696F6E2070617291
:10471000616D6574657220726571756573743A2098
:10472000307825780000000064300020436F6E6E02
:104730006563746564000000A6C507004661696C86
:1047400075726520746F2075706461746520636F85
:104750006E6E656374696F6E20706172616D6574F1
:104760006572733A203078257800000094CC0700F9
:10477000526563656976656420424C455F474150E8
:104780005F4556545F444154415F4C454E47544841
:104790005F5550444154455F524551554553542E41
:1047A00000000000526563656976656420424C45EF
:1047B0005F4741505F4556545F444154415F4C450B
:1047C0004E4754485F555044415445202825752C88
:1047D000206D61785F72785F74696D652025752939
:1047E0002E000000526563656976656420424C4581
:1047F0005F4741505F4556545F5345435F504152B8
:10480000414D535F52455155455354004343434432
:1048100020666F72207365727669636520636861D4
:104820006E67656420697320307825303478000025
:10483000526563656976656420424C455F47415027
:104840005F4556545F5048595F5550444154452088
:104850002852583A25642C2054583A25642C207349
:1048600074617475733A25642900000052656365AC
:104870006976656420424C455F4741505F45565418
:104880005F5048595F5550444154455F524551551A
:104890004553542E00000000436F756C64206E6F0A
:1048A000742068616E646C65206F6E5F6374726CF7
:1048B0005F70745F77726974652E206572725F63D2
:1048C0006F64653A2030782530347800526563652E
:1048D0006976656420424C455F4741505F455654B8
:1048E0005F5345435F494E464F5F524551554553CF
:1048F0005400000046696E69736865642068616EE3
:10490000646C696E6720636F6E6E207365632075DB
:104910007064617465000000007800F00100704769
:1049200038B50020009002F043FC00282DD1174834
:104930001749184A401AC108042000EB01400446F8
:1049400015A104F09DFA134813DF00281DD120465D
:1049500019A104F091FA04F071FE002815D16846FF
:1049600004F0D2FC002810D1204619A104F084FAEA
:104970006946012004F0D2FC002806D120461AA185
:1049800004F07AFA684604F061FD38BD40DB0700A8
:1049900038DB07000020070053657474696E6720D8
:1049A000757020766563746F72207461626C653A0D
:1049B0002030782530387800456E61626C696E670A
:1049C00020536F66744465766963652E00000000AD
:1049D000436F6E6669677572696E6720424C452049
:1049E000737461636B2E0000456E61626C696E6763
:1049F0002074686520424C4520737461636B2E00FF
:104A000013B90378012B01D003F00EB801207047D1
:104A10000022C32100F5187000F0CCB92DE9F04355
:104A2000A1B00446DDE9289620200F462090984644
:104A30001546782102A8FDF70EFD41212046FDF71D
:104A40000AFDB7F8940005EB051107EB8101A842B8
:104A500001D991F896602670320033D0012A0DD02A
:104A60001B481C4D0123401BC00803EB0045022AD4
:104A70000CD0032A20D0284617A117E0002249466F
:104A8000404600F097F9C4F801001BE020A9601C23
:104A9000CDE900014B464246184902A801F052FEFA
:104AA00080B104F0FDFE0246284615A104F0E8F9A5
:104AB000002021B0BDE8F083B1F89820601C9A3145
:104AC000FDF7B0FC4A464146204602F0ADFFF0E754
:104AD00068DB070038DB0700496E76616C6964208B
:104AE000626F6F742076616C69646174696F6E20A7
:104AF000747970653A20256400000000B8C307008F
:104B00006E72665F63727970746F5F686173685FFD
:104B100063616C63756C6174652829206661696CDA
:104B200065642077697468206572726F72202573DE
:104B30000000000010B504460A480B49401AC0089E
:104B4000042101EB004009A104F096F94FF00000A8
:104B500034B10C490870BDE810400B4802F01EBD8E
:104B600000F084FB88DB070038DB070052657365C3
:104B70007474696E6720626F6F746C6F61646572C4
:104B80002E000000E82A00206D5207002DE9FC41AC
:104B90000646C0074FF000050ED0104F002401223A
:104BA000385D009500231146019503F081FE641CD9
:104BB000042CF4D300F064F8B0070DD5074E0024A0
:104BC000361D0022305D032300951146019503F048
:104BD0006FFE641C042CF4D3BDE8FC81A6C307005F
:104BE00010B50446042803D305A14720FFF748F970
:104BF0000E480121005DBDE8104003F0EFBE00004B
:104C00002E2E5C2E2E5C2E2E5C2E2E5C2E2E5C63A9
:104C10006F6D706F6E656E74735C626F61726473DA
:104C20005C626F617264732E63000000A6C30700AC
:104C300010B50446042803D305A14120FFF720F94D
:104C40000E480021005DBDE8104003F0C7BE000023
:104C50002E2E5C2E2E5C2E2E5C2E2E5C2E2E5C6359
:104C60006F6D706F6E656E74735C626F617264738A
:104C70005C626F617264732E63000000A6C307005C
:104C800010B500242046FFF7ABFF641C042CF9D3B9
:104C900010BD00002DE9F84F0546861C00208DF858
:104CA000000091460F464FF0010A6846FFF758F89A
:104CB0001C4C60683860D4E901011B4F401A396808
:104CC000081A41F21C0104EB01080EE001214046E4
:104CD00000F0E7FF00F03CFE0146404600F0E1FF37
:104CE000D4E90101401A3968081A401C8642EDD8FF
:104CF000B9F1000F03D0052065F3891002E006200A
:104D000065F39F5061683A68114004EB8101C86007
:104D10006068304460609DF80000FFF76DF8504611
:104D2000BDE8F88FD8520020982B002010B54368BA
:104D30009C18446021B905E013F8010B01F8010B40
:104D4000521EF9D2012010BD70B50D4604460A2945
:104D500002D10D21FFF7F8FFA0682268411CA16075
:104D60001554D4E90101814204D32046BDE87040C6
:104D700003F0A6BA70BD0000044881684068814213
:104D800001D101207047002070470000D852002058
:104D900010B5040003D10549F020FFF771F804486D
:104DA000C16B6160006CA06010BD0000DCCD07002D
:104DB000C0470020F0B54FF0FF3622B11268D24351
:104DC00000230A4D0DE03246FAE7C45C6240082435
:104DD000D70700D037462F4087EA5202641EF7D12A
:104DE0005B1C8B42F1D3D043F0BD00002083B8EDB3
:104DF00010B504460068401C07D0204606F032FC7F
:104E00002168814201D1012010BD002010BD0000A9
:104E100010B5104C90B06078002818D101F0F6FC65
:104E200018B10D49DB20FFF72BF820220B4968460B
:104E300001F00CFD40236A4609490A4801F042FC92
:104E400018B10549E520FFF71BF80120607010B08C
:104E500010BD0000602B0020BCD1070060C307001C
:104E60006C4E0020D0C30700F0B5146906468DB023
:104E700020681546271DE0B1022920D00A200090A5
:104E80006B4609AA304606F04BF900280FD009A955
:104E900001A8009A05F070FE01AE96E80F0005AE7D
:104EA00086E80F00236869683A4605A898470DB060
:104EB000F0BD0DB03046BDE8F04005F0D1BE69460A
:104EC000304605F063FE0028F1D0236869683A4651
:104ED000684698470028EAD002980028F5D1019842
:104EE00070600120E3E753689B7813F0C00303D0A0
:104EF000402B03D00020704700F002B8FFF7B4BF8A
:104F00002DE9FF410B465168064614468878334D1B
:104F100000F00F0210F0300055F8225006D0102893
:104F200006D0202808D0302856D13EE022694DE036
:104F300061690120087047E0022B28D1042A26D895
:104F40004FF0010869463046676905F01FFE0028EA
:104F50001AD009E00B89226903FB00226846A847A2
:104F600070B13888401C3880029820B16168388858
:104F70004A899042EED301987060029860BB02E0CB
:104F80004FF00008F7E7404604B0BDE8F081D4E9EF
:104F900004300F890288498907FB02338A421BD2F9
:104FA000521C02801A46616810E008886169072A6D
:104FB000088009D1606801892069FDF74CFA6068B2
:104FC0002169C06805F0FDFD2269616804B03046C2
:104FD000AC46BDE8F04160470020D5E758CA07005D
:104FE00038B51E4901200A68D20301D5000408E043
:104FF0001B490A6802F0F902A92A04D1086800F0E6
:10500000560008600020FEF789FD1649164A891AE5
:10501000C908042202EB0144A0B11920009068469F
:1050200003F09EFCD0F810050099C84010F0010F65
:105030000BD00B48001F006800F0F900B12807D022
:10504000002038BD204609A104E0204610A101E05F
:10505000204617A103F010FF012038BD00040040D6
:105060002005004088DB070038DB07004446552058
:105070006D6F646520626563617573652061707032
:10508000206973206E6F742076616C69642E000055
:10509000444655206D6F6465207265717565737443
:1050A00065642076696120627574746F6E2E0000ED
:1050B000444655206D6F6465207265717565737423
:1050C0006564207669612047505245475245542E09
:1050D00000000000FEB519490446086808B1401EEA
:1050E00008601748174AD4E90153801AC0080422FF
:1050F00002EB004022789DB10E6821690296CDE94D
:1051000000312B46012A16D00FA211A103F0DAFEBE
:105110006169002911D0E06803B0BDE8F04008479C
:1051200009680091012A04D007A218A103F0B7FE74
:10513000EEE720A2F9E71FA2E7E7FEBD442B00201F
:1051400048DB070038DB070065726173650000000B
:10515000466C617368202573206661696C65642004
:105160002830782578293A20616464723D25702CB6
:10517000206C656E3D307825782062797465732CDB
:105180002070656E64696E6720256400466C6173EB
:105190006820257320737563636573733A206164B7
:1051A00064723D25702C2070656E64696E672025E1
:1051B00064000000777269746500000010B508286B
:1051C0001BD2DFE800F004121A1A1A041A04012094
:1051D000FFF7DCFC0020FFF72BFD0120FFF728FD87
:1051E000BDE810400220FFF7FBBC0120FFF7F8FCF0
:1051F000BDE810400220FFF71BBD10BD10B50446EE
:10520000801E062810D2DFE800F00D03030F090905
:105210000A494FF4701000F087FF05E00120FFF706
:1052200089FC01E002F046FA05484168002903D0F4
:105230002046BDE81040084710BD0000D1560700C9
:10524000E82A002010B50446062801D0072C02D118
:10525000002002F02BFB04480168002903D02046FF
:10526000BDE81040084710BD282B002003F0BCFE0D
:1052700003F092FC0028FBD1BFF34F8F0548016873
:10528000054A01F4E06111430160BFF34F8F00BF95
:10529000FDE700000CED00E00400FA0510B5002168
:1052A000024800F014FD80F3100010BDF4620020ED
:1052B0002DE9FC4180461F4615460E4600240D4848
:1052C00000F0ECFC38B11120BDE8FC8106EB0430A5
:1052D00003F0B4FF641CAC42F8D1064800F0D5FCE2
:1052E000CDE90057334600220221404600F02AF85B
:1052F0000020E9E7802B00202DE9F843104D0F46F0
:1053000080461E4691466946286800F092FC0400DB
:1053100014D01C21FDF79FF801202071C4F81490CF
:10532000380BC4F80080C4E902606946286800F0C0
:10533000A1FC05F0D5FE0020BDE8F8830420FBE7C2
:1053400024C707002DE9F04387B00446DDE90E8944
:1053500080681D4616460F4600280BD01821684667
:10536000FDF779F802A88DF8007080E86003A16865
:105370006846884707B0BDE8F08330B5044600684A
:1053800087B00D46806800281FD018216846FDF7B9
:1053900062F80195A0680590207910B1012810D11C
:1053A00007E001208DF8000020690290E06803907A
:1053B00005E002208DF80000E068000302906069BB
:1053C0000490206881686846884707B030BD0B2884
:1053D00003D30B38C0B200F009B87047024900226D
:1053E00008780A7070470000482B002001490870B7
:1053F0000B207047482B002001490120087070479E
:10540000E82A00200149012008707047242B002061
:1054100070B515460E46040004D107494FF42C70B0
:10542000FEF72EFD2A46314604F17200BDE87040B9
:10543000012302F04BBB0000BCD1070010B50400F3
:1054400003D10E49DB20FEF71BFD207818B90B496C
:10545000DC20FEF715FD94F85500094938B1012804
:1054600005D06068C968884205D9012010BD606810
:1054700089688842F9D24FF0000010BD04D20700BD
:10548000C04700203EB59DF8080020F00F00401CEA
:1054900020F0F00010308DF8080068466DDF00281D
:1054A0002BD19DF80100401C8DF8010068466CDF8F
:1054B000002822D111481349007A82071048A0EB36
:1054C00001004FEAD0004FF0040101EB004008D585
:1054D0000D4C0EA1221DA36903F0D9FC211DA0696A
:1054E00004E013A103F0C8FC19A1072082B202A8AE
:1054F0007CDF002801D118487ADF3EBD2C2B00202C
:1055000040DB070038DB0700483000205365747427
:10551000696E6720616476206E616D653A2025733F
:105520002C206C656E6774683A20256400000000CA
:105530005573696E672064656661756C742061647B
:10554000766572746973696E67206E616D650000BF
:105550004466755461726700A6C507002DE9FC5FBB
:10556000164607463A4A3B481D46101A04224FEA9F
:10557000D00902EB09408B468246B94205D136A1DB
:1055800003F07AFC0020BDE8FC9F04D236494FF0BE
:105590004F00FEF775FC1DB933495020FEF770FC33
:1055A0002EB1380503D030495320FEF769FCABEB30
:1055B0000700040B03D12C495720FEF761FC0020A3
:1055C000009006F6FF704FEA103800F0D1FFA542B8
:1055D00039D22C4637E0A04503D83546CDF80480B3
:1055E00001E02503019400223846019901F062FC94
:1055F0000028C8D150463B465A461CA1009503F0EE
:105600004EFC681E00F003002A1A00235946384653
:10561000D21C01F005FD0028B5D101991C48A8EB6A
:105620000108761B016B2F4429440163AB44002021
:1056300002F028F9009030B1012101EB094015A1D9
:1056400003F01AFC01E0002EC5D100989BE7000092
:1056500088DB070038DB07004E6F20636F7079200E
:105660006E65656465640000A0CB0700436F7079C8
:10567000696E67203078257820746F20307825781F
:105680002C2073697A653A20307825780000000074
:10569000C04700204661696C656420746F20777292
:1056A00069746520696D61676520636F7079696EE3
:1056B000672070726F677265737320746F207365F3
:1056C0007474696E677320706167652E0000000056
:1056D0000748084910B5401AC008032101EB0040F3
:1056E00005A103F0C9FBBDE810400120FFF722BA75
:1056F00088DB070038DB0700496E616374697669EF
:1057000074792074696D656F75742E00014941606C
:1057100000207047F8C6070010B50B4941600B48E0
:1057200000F0BCFA68B903F0DBFF08491C234FF412
:10573000EE7208740448A1F5EE71001F006800F0D5
:1057400065FA002010BD000028C707002C5100207A
:105750002DE9FC5F0E008346DDE90C47C6F1000031
:1057600098469246814600D40846012503E000BFD2
:1057700090FBFAF06D1C5045FADAA84500D9454671
:1057800024B1002E01DB780700D5641EB80702D5CE
:10579000B8F1000F0AD0F80708D13CB1A54205D2F4
:1057A00020215846641EFFF7CFFAF6E7002E02DAF2
:1057B0004E462D2102E0780703D52B215846FFF7EE
:1057C000C3FA07F0030002280BD1B8F1000F08D18B
:1057D0003CB1A54205D230215846641EFFF7B4FA09
:1057E000F6E7CDE90047434652463146584606F0B3
:1057F00015FCBDE8FC9F024600201268530713D534
:1058000002F00300012802D002280CD105E0C2F307
:1058100083100B68801C184404E00223086803EB23
:10582000925210440860012070470000024800684E
:10583000002800D001207047802B00200248007A09
:10584000002800D0012070472C51002038B54FF4BB
:1058500040521B49536800F500508B4204D0446805
:105860008C4201D1012400E000248B4226D1436800
:105870008B4223D11178142901D9526900E000220A
:105880001049B2FBF1F30278142A01D9406900E013
:105890000020B0FBF1F0834203D001240AA2009063
:1058A00002E000240AA200900B480C49401AC008EC
:1058B000032101EB00400AA103F0F1FA204638BDB4
:1058C000DBE5B15140420F006D616A6F720000006C
:1058D0006D696E6F7200000068DB070038DB07003F
:1058E000536F66744465766963652075706461748E
:1058F0006520697320612025732076657273696F56
:105900006E207570646174652E2043757272656EC9
:10591000743A2025642E204E65773A2025642E00A7
:1059200070B5054608680C464A68866828463146C0
:1059300005F068F86068286104F10C006861B078CF
:105940000221B1EB901F01D1241D2C6170BD704765
:105950002DE9FF410026274800F09DF92548001F4A
:10596000074600F098F9244C2449A06800900D687F
:1059700000E000986946284004EB80000C30FFF7F7
:105980003AFF0028F5D101AA009901EA050304EBCA
:105990008303491CDB6842F82030401C0091022838
:1059A000F2D3019800F0030001281AD002280ED08B
:1059B00013A14FF4C270FEF763FA384600F068F99D
:1059C00008B10098A06004B03046BDE8F0810198AD
:1059D000032101EB90500099BDF80A6001EB9000A3
:1059E00005E00198BDF80A60C0F3831008440090F8
:1059F000E3E70000F0620020D8520020982B00203E
:105A00002E2E5C2E2E5C2E2E5C2E2E5C2E2E5C639B
:105A10006F6D706F6E656E74735C6C6962726172CB
:105A20006965735C6C6F675C7372635C6E72665FF2
:105A30006C6F675F66726F6E74656E642E630000D4
:105A400000F06AFD4FF48051002000F08DFBC8B9D2
:105A50001548C0F5FC2100F087FB98B900211348D8
:105A600003F096FA03F082F811481249401AC4086C
:105A7000032000EB044010A103F0FEF9114800F0F0
:105A800079FC08B1FEF72AF803F086F80028FBD16C
:105A9000012000EB04400CA103F0EEF903F07CF8C8
:105AA0000028FBD1EEE7000000200700516107004D
:105AB00088DB070038DB0700496E73696465206D79
:105AC00061696E00BD5107004166746572206D61A9
:105AD000696E2C2073686F756C64206E65766572D4
:105AE00020626520726561636865642E00000000B5
:105AF0002DE9F05F1E46DDF828B091468A46040085
:105B000003D124A1B620FEF7BBF9B4F80680607972
:105B100008FB00F8A8F10408464503D31DA1C420E2
:105B2000FEF7AEF9E788301DB0FBF7F1B0FBF7F2F6
:105B300007FB1200D9F80050AA19424501D9A8EB79
:105B40000605C9F8005001E02468491E0029FBD170
:105B50003E1A8846AE4215D817E000BF2044001D0B
:105B60000AEB0803BBF1000F324602D0014618468B
:105B700000E01946FCF756FC00202468AD1BB04439
:105B8000AF4201D92E4600E03E46002DE6D1BDE8E9
:105B9000F09F00002E2E5C2E2E5C2E2E5C2E2E5C96
:105BA0002E2E5C636F6D706F6E656E74735C6C69C6
:105BB000627261726965735C6D656D6F626A5C6E5D
:105BC00072665F6D656D6F626A2E630030B5024666
:105BD00051B103F0F1F90021074C08E034F821300D
:105BE0001568AB4202D11160002030BD491C8142D2
:105BF000F4D3052030BD00000000000010B5FCF714
:105C000056FB08B1002010BD112010BD10B531B1F8
:105C1000B2FBF3F403FB14241CB1092010BD0E20C9
:105C200010BD01600021416081608281C38108460E
:105C300010BD70B50C460546FCF7EEFA002802D000
:105C400021882868084470BD10B50A8849888A42AE
:105C500003D1FCF723FB012010BD002010BD70B55F
:105C60000C460546FCF7FDFA002802D0618828683A
:105C7000084470BD10B50A8849888A4203D1FCF7F0
:105C8000E7FA012010BD002010BD002100F00FB880
:105C9000002100F012B8012100F01EB8012100F02F
:105CA00011B808B56A46FCF74EFB009808BD08B568
:105CB0006A46FCF72EFB009808BD08B56A46FCF75B
:105CC00028FB08BD08B56A46FCF716FB08BD08B5F9
:105CD0006A46FCF705FB08BD08B56A46FCF70CFBF5
:105CE000009808BD08B56A46FCF73AFB009808BD65
:105CF00038B5040004D115A14FF49270FEF7C0F836
:105D000000258DF800506846FEF72AF82068626882
:105D10000168914214D9491E01600D781CB919A17E
:105D2000E820FEF7ADF8208AE16805FB0015206841
:105D3000217A0278891A0279C9B28A4200D20171A5
:105D40009DF80000FEF758F8284638BD2E2E5C2E30
:105D50002E5C2E2E5C2E2E5C2E2E5C636F6D706F73
:105D60006E656E74735C6C69627261726965735C96
:105D700062616C6C6F635C6E72665F62616C6C6FAB
:105D8000632E63002E2E5C2E2E5C2E2E5C2E2E5C3F
:105D90002E2E5C636F6D706F6E656E74735C6C69D4
:105DA000627261726965735C62616C6C6F635C6E78
:105DB00072665F62616C6C6F632E630038B50C466F
:105DC000050004D112A140F24710FEF759F824B99A
:105DD0000FA14FF4A470FEF753F800208DF80000D7
:105DE0006846FDF7BDFF1DB91749F520FEF748F8D5
:105DF000E8682A68211A288AB1FBF0F11068431C70
:105E0000136001709DF80000FDF7F6FF38BD00003B
:105E10002E2E5C2E2E5C2E2E5C2E2E5C2E2E5C6387
:105E20006F6D706F6E656E74735C6C6962726172B7
:105E30006965735C62616C6C6F635C6E72665F62F5
:105E4000616C6C6F632E6300845D070010B5040005
:105E500002D0206830B901E00E2010BD19A1FF204A
:105E6000FEF70EF8606820B916A14FF48070FEF7B7
:105E700007F8A06820B913A140F20110FEF700F85E
:105E8000E06820B90FA14FF48170FDF7F9FF208A77
:105E900020B90CA140F20310FDF7F2FF207A6168EF
:105EA0002268401AC0B2116004E0226811684B1CDD
:105EB00013600870401EC0B2F7D22168002008713C
:105EC00010BD00002E2E5C2E2E5C2E2E5C2E2E5C25
:105ED0002E2E5C636F6D706F6E656E74735C6C6993
:105EE000627261726965735C62616C6C6F635C6E37
:105EF00072665F62616C6C6F632E63002DE9F04126
:105F0000184819494FF48052401AC708042000EB82
:105F10000745164615A1284602F0B2FF4FF0E024CF
:105F2000D4F8802128461FA104F5C07402F0A8FF10
:105F300060172060C4F800016060C4F8040101F03B
:105F400043F928B1012000EB074021A102F094FFA2
:105F500002F022FE0028FBD13046BDE8F04100F0FF
:105F600053B8000088DB070038DB070052756E6EFF
:105F7000696E67206E72665F626F6F746C6F6164CA
:105F800065725F6170705F73746172742077697499
:105F90006820616464726573733A20307825303804
:105FA0007800000044697361626C696E6720696EF5
:105FB00074657272757074732E204E5649432D3E6F
:105FC000494345525B305D3A203078257800000027
:105FD0004661696C65642072756E6E696E67206ECD
:105FE00072665F6466755F6D62725F6972715F662B
:105FF0006F72776172645F616464726573735F73FB
:10600000657428290000000070B506462648C0F5D2
:10601000FE2100F0A9F8040024482549A0EB010066
:106020004FEAD0004FF0010101EB004507D02846B0
:10603000224620A102F024FF2046FDF74FFD00F08C
:10604000AFFC014629488069421EC2F30B02801A48
:106050000144002001F6FF7100F086F8040004D02E
:106060002846224622A102F00BFF201E01D0FDF798
:1060700035FDEFF30580C105D6E90045C90D4FF0A8
:10608000000080F3148880F3108880F3118880F377
:10609000138803D023495820FDF7F2FE84F30888C3
:1060A000AC46BDE8704060470020070088DB070071
:1060B00038DB0700436F756C64206E6F742070725C
:1060C0006F7465637420626F6F746C6F6164657266
:1060D00020616E642073657474696E6773207061EB
:1060E0006765732C20307825782E0000C04700208B
:1060F000436F756C64206E6F742070726F7465638B
:106100007420536F667444657669636520616E64BC
:10611000206170706C69636174696F6E2C203078D7
:1061200025782E0004CB070070B5084D04460E46B6
:10613000686805F02BFF002C06D0324621466868BF
:10614000BDE8704005F014BF70BD0000F42A0020C7
:106150000348D0F804050349097B00EB0160704750
:1061600000400240F42A002030B50A0502D1B0F503
:10617000FE2F01D9072030BD094C2268082A01D31F
:10618000042030BD074B03EB0213C3F80008C3F82B
:1061900004180220C3F80808521C0020226030BDF9
:1061A000F02A002000E001402DE9F0413A483B4947
:1061B000384E401AC508042000EB0540002704466D
:1061C00037A102F059FEB06801280ED0A52813D0DF
:1061D000AA2818D0AC281ED0032000EB054039A116
:1061E00002F04AFE0020BDE8F08120463CA102F00A
:1061F00043FEFDF7BFFB0CE020463CA102F03CFE55
:1062000004F0EEFF0DE020463BA102F035FEFDF765
:1062100041FE024607E020463AA102F02DFE05F0BD
:10622000ADF8024601271D491B4B0120591AC90828
:1062300000EB014522B1284636A1B36802F027FEE3
:10624000304600F0D1FBDFF80081002188F8001013
:106250003E4801F017FB064698F8000020B93C497B
:1062600040F2A510FDF70CFE2EB1284639A102F030
:1062700003FE0320B7E70120002FB4D005492439DD
:10628000096A0129AFD12046394902F0F5FD022003
:10629000A9E70000E447002088DB070038DB07009F
:1062A000456E746572206E72665F626F6F746C6F9C
:1062B000616465725F66775F616374697661746556
:1062C000000000004E6F206669726D776172652074
:1062D000746F2061637469766174652E000000003C
:1062E00056616C69642041707000000056616C69F1
:1062F000642053440000000056616C696420424CE5
:106300000000000056616C6964205344202B204239
:106310004C00000041637469766174696F6E206699
:1063200061696C65642077697468206572726F7248
:10633000202564202862616E6B20636F64653A20BB
:106340003078257829000000242B00200554070010
:10635000A0CB0700436F756C64206E6F742077725A
:106360006974652073657474696E67732E0000002C
:1063700038CC07002DE9F843044641484149401A0A
:10638000C108042000EB014005463FA102F074FD66
:10639000434F19207C600090684602F0E1FA009AB1
:1063A000404900EB82004FF00008C0F8001740465B
:1063B00001F0FAF800284CD1FFF7F6FE314A304BD5
:1063C00001219A1AD20801EB024420B101281BD006
:1063D00002283ED105E04FF47016FEF701FE10B919
:1063E00034E04FF4A02600F0C3F82F4A20211820F3
:1063F000FDF7A0FC08B1FDF771FB2C48016801F026
:10640000F901B12904D007E00120FEF793FB31E048
:10641000016801F04E01016000F09EFEC8B92449F8
:106420003046FFF781FE234800F04AFE88B928462F
:1064300021A102F021FD00BF00F086F8FDF75AFC13
:1064400002F0AAFB0028F7D141DFF5E701F032F8AE
:1064500010B10320BDE8F88387F800801A4801F0E6
:106460009DF8387820B919A140F20620FDF708FD03
:10647000FFF744FD204625A102F0FEFCE9E70000FD
:1064800088DB070038DB0700496E206E72665F62AA
:106490006F6F746C6F616465725F696E6974000020
:1064A000E82A00200C000300082C00201C050040F6
:1064B000D1560700FD510700456E746572206D616D
:1064C000696E206C6F6F7000F95307002E2E5C2EE2
:1064D0002E5C2E2E5C2E2E5C2E2E5C636F6D706FEC
:1064E0006E656E74735C6C69627261726965735C0F
:1064F000626F6F746C6F616465725C6E72665F620E
:106500006F6F746C6F616465722E6300556E726597
:1065100061636861626C650010B540F6F8700168EF
:10652000491C02D1074902F0A1FE40F6FC70016847
:10653000491C05D1BDE810404FF4FC2102F096BE85
:1065400010BD00000020070010B503F0F9F9002885
:1065500003D0BDE8104005F07BBE10BD034A936830
:106560000A4601469860184605F002BDF42A00204C
:106570002DE9F0411A4E307800282ED103F0E0F9D1
:106580001849194A0127891AC908032202EB014553
:1065900000281DD0154804682846224614A102F0A0
:1065A0006FFCA4F54864962C00DA962405F050FEA2
:1065B0002846224615A102F063FC21492046FFF738
:1065C000CDFF4FF0E0214FF48030C1F8000103E02F
:1065D00028461CA102F050FC3770BDE8F081000095
:1065E000252B002038DB070038DB070004050140BD
:1065F00057445420656E61626C6564204352563A7C
:106600002564207469636B73000000005374617229
:1066100074696E6720612074696D65722028256435
:10662000207469636B732920666F722066656564E8
:10663000696E67207761746368646F672E0000007D
:106640008DC20700574454206973206E6F74206513
:106650006E61626C6564000040688068004710B538
:1066600042680830527900F0F1F8002010BD2DE9A1
:10667000F04399B01C4690460D460846DDF88090E0
:10668000FFF7EAFF6E6807467079A04200D804461B
:106690002246414611A800F015F97279494601A831
:1066A00000F0D4F801AB224611A905F108000097CB
:1066B000FCF78AF818B1002019B0BDE8F08348F261
:1066C0004250F9E770B516460C46054600F0E2F870
:1066D00000280ED1AA791946304600F0E8F80028C3
:1066E00007D131462046FFF7BAFF002801D1014902
:1066F000216070BD7052464D2DE9F8430C46DDE92E
:1067000008578146984616460D49204600F0B6F8CF
:10671000002810D16068394640794200284600F0D0
:10672000C6F8002807D146B14346324621464846BE
:106730000095FFF79CFFBDE8F88348F21050FAE798
:106740007052464D2DE9F0411D46DDE9068716469B
:10675000044600F02DF800280DD12A463146204687
:1067600000F03CF8002806D13A4641462046BDE8F4
:10677000F04100F002B8BDE8F08170B515460E4654
:10678000044605F055FD002807D13EB16068296830
:10679000C268914205D248F2145070BD48F21350BD
:1067A00070BD83682A4631462046BDE870401847D0
:1067B00010B550B161B141600968044688470028AE
:1067C00002D105482060002010BD48F2015010BDE4
:1067D00048F2105010BD00006E52464870B5154684
:1067E0000E46044605F024FD00280BD146B155B1F4
:1067F00060682A46314643682046BDE87040184725
:1068000048F2105070BD002070BD00002DE9F0412D
:106810000B480C4D0C4F401BC6080120387000245B
:1068200006E000BF55F834008047002805D1641CFD
:10683000B442F7D3022038700020BDE8F081000098
:106840000000000000000000262B002070B5144658
:106850000D46064600F036F8291930192246BDE8E3
:10686000704000F02FB870B50C46054600F064F893
:1068700028192146BDE8704000F05EB828B10068D4
:10688000884205D048F24050704748F21050704797
:106890000020704728B139B10022C1E9002010461C
:1068A000704748F21050704748F21350704720B1BB
:1068B000914205D048F21150704748F2105070478D
:1068C0000020704770B516460C46050003D10AA19A
:1068D0004520FDF7D5FA1CB907A14620FDF7D0FAEF
:1068E000A919491E04E000BF14F8010B01F80109C1
:1068F000A942F9D270BD00002E2E5C2E2E5C2E2EE9
:106900005C2E2E5C2E2E5C636F6D706F6E656E74E8
:10691000735C6C69627261726965735C63727970D1
:10692000746F5C6E72665F63727970746F5F7368A8
:10693000617265642E63000070B50D46040003D1DA
:1069400007A13320FDF79CFA6019401E05E021786D
:10695000027804F8012B00F80119A042F7D270BDAB
:106960002E2E5C2E2E5C2E2E5C2E2E5C2E2E5C632C
:106970006F6D706F6E656E74735C6C69627261725C
:106980006965735C63727970746F5C6E72665F6365
:10699000727970746F5F7368617265642E63000052
:1069A0004FF44050074A4168914207D18068411E28
:1069B000C1F30B01401A00F6FF7070474FF480508E
:1069C00070470000DBE5B15100B5FFF7E9FF05496D
:1069D00089690A18401E0844C0F30B00101A00F61B
:1069E000FF7000BDC0470020002101604160816050
:1069F0000148016370470000C04700202DE9FF4FA8
:106A00008B466948694981B0401AC108042000EBEF
:106A10000144009166A1204602F02EFA20466CA1A6
:106A2000019A02F02DFABBF1000F01D06EA200E036
:106A30006FA2204670A102F023FA039808B16AA25F
:106A400000E06BA2204671A102F01AFA049808B186
:106A500065A200E066A2204670A102F011FA4FF490
:106A6000405041687348814201D15FA200E060A2BA
:106A7000204671A102F004FA204673A102F0FCF94D
:106A8000754D204675A1AB692A6A02F000FA2046CE
:106A90007AA16B6AEA6A02F0FAF94FF00009DFF8AE
:106AA000FCA10CE0012650B1012812D0B9F1020F6F
:106AB0001ED07B49AC20FDF7E3F900201AE0FFF778
:106AC00083FF8046039888B16348006A01280BD091
:106AD0000CE0FFF765FF8046049828B94FF440505A
:106AE00041685448814201D0012604E0002602E0BA
:106AF0004FF480508046D04503D96949B120FDF755
:106B0000BFF968490198A1EB0801A1F50051814244
:106B100001D2012700E0002747EA0B0520464A463C
:106B200061A102F0ADF92046424662A102F0A8F947
:106B30000FB12DA200E02EA2204664A102F0A0F920
:106B40000EB129A200E02AA2204666A102F098F91F
:106B50000DB125A200E026A2204667A102F090F91F
:106B6000B54308D0B9F1020F05D209F10100C0B256
:106B70008146022896D957B10098022101EB0040C6
:106B800062A102F079F9042005B0BDE8F08FB9F1F7
:106B9000000F07D0204668A102F06EF92E48183089
:106BA000FFF722FF0020EFE788DB070038DB070054
:106BB000456E746572206E72665F6466755F6361B0
:106BC0006368655F707265706172652829000000F6
:106BD00072657175697265645F73697A653A2030B0
:106BE0007825782E000000007472756500000000A2
:106BF00066616C736500000073696E676C655F6247
:106C0000616E6B3A2025732E000000006B65657085
:106C10005F6170703A2025732E0000006B6565700F
:106C20005F736F66746465766963653A2025732EB9
:106C300000000000DBE5B15153445F50524553451D
:106C40004E543A2025732E0042616E6B20636F6EA6
:106C500074656E74733A0000C047002042616E6B29
:106C6000203020636F64653A203078253032783ADE
:106C70002053697A653A20307825780042616E6B3E
:106C8000203120636F64653A203078253032783ABD
:106C90002053697A653A2030782578000000070093
:106CA0007CCF070000200700706173733A202564D1
:106CB0002E00000063616368655F616464726573E0
:106CC000733A20307825782E0000000063616368F5
:106CD000655F746F6F5F736D616C6C3A2025732E06
:106CE000000000006B6565705F6669726D776172A8
:106CF000653A2025732E000064656C6574655F6DD0
:106D00006F72653A2025732E0000000041626F7299
:106D100074696E672E2043616E6E6F7420666974AD
:106D2000206E6577206669726D77617265206F6E7F
:106D30002064657669636500496E76616C6964619B
:106D400074696E67206170702E00000070B50C468B
:106D5000050004D121494FF4AC70FDF791F824B936
:106D60001E4940F25910FDF78BF81D481D4B29783C
:106D7000C01A0422C00802EB0040092927D2DFE82C
:106D800001F02605260B15261B260F002146284656
:106D9000BDE8704002F0E8BD13A102F06DF811E00B
:106DA00021462846BDE8704002F082BE21462846B2
:106DB000BDE8704002F01ABE14A102F05DF84FF475
:106DC0000070E0602046BDE87040FDF7E1BFBDE81F
:106DD000704002494FF4BC70FDF752B8DCCD07009B
:106DE00050DB070038DB070048616E646C65204E9D
:106DF00052465F4446555F4F505F4352435F47459D
:106E0000542028636F6D6D616E64290048616E6463
:106E10006C65204E52465F4446555F4F505F4F426F
:106E20004A4543545F53454C4543542028636F6D96
:106E30006D616E642900000070B50E46040004D137
:106E40001B4940F27520FDF71BF826B9184940F29E
:106E50007620FDF715F820780125092820D2DFE8F3
:106E600000F01F051F0F141F1A1F0A00314620468D
:106E700002F004FF19E03146204603F055F914E012
:106E80003146204602F0BCFE0FE03146204602F0BB
:106E9000FFFF054609E03146204603F0F9F804E01B
:106EA000034940F29720FCF7EBFF284670BD000035
:106EB000DCCD07002DE9F843134C07460D4620684A
:106EC0000090124812499046401AC608042000EB70
:106ED00006402B463A460FA101F0E1FF43462A4601
:106EE00039461C4801F040FB050009D0022000EBA8
:106EF00006402A4618A101F0C3FF2846BDE8F883E2
:106F00002068401C2060F8E7442B002048DB070085
:106F100038DB07006E72665F6673746F7261676557
:106F20005F657261736528616464723D30782570B5
:106F30002C206C656E3D2564207061676573292C7B
:106F40002071756575652075736167653A202564E4
:106F500000000000F42B00206E72665F6673746F91
:106F6000726167655F657261736528292066616972
:106F70006C65642077697468206572726F72203066
:106F80007825782E000000000C490D4A10B5891AAA
:106F9000C908042202EB01420028104604D009A1CE
:106FA00001F06AFF114903E011A101F065FF1A49E0
:106FB000BDE810400022194801F036BB48DB07004D
:106FC00038DB0700496E697469616C697A696E67BC
:106FD000206E72665F6673746F726167655F73645B
:106FE000206261636B656E642E00000034C7070089
:106FF000496E697469616C697A696E67206E726640
:107000005F6673746F726167655F6E766D63206231
:1070100061636B656E642E0004C70700F42B0020CB
:107020002DE9FC47154C80460F4620681549CDE9EF
:10703000002013489946401AC6081546042000EB64
:1070400006403B464246104901F032FF2B463A4685
:1070500041460E48CDF8009001F0AEFB050009D086
:10706000022000EB06402A4609A101F009FF28464C
:10707000BDE8FC872068401C2060F8E7442B002016
:1070800048DB070038DB070024CD0700F42B002085
:107090006E72665F6673746F726167655F7772693F
:1070A00074652829206661696C6564207769746855
:1070B000206572726F7220307825782E00000000F3
:1070C00070B51149086011481149401AC5080320DC
:1070D00000EB05400FA101F0CFFE0020FEF7B2F853
:1070E000114800F041FC040008D0012000EB0540ED
:1070F00022460EA101F0C4FE204670BDBDE87040DE
:10710000094800F0A7B80000282B002088DB070002
:1071100038DB0700456E746572696E67204446551A
:10712000206D6F64652E000045520700436F756C3B
:1071300064206E6F7420696E6974616C697A652071
:10714000444655207472616E73706F72743A2030C9
:1071500078253038780000000648074910B5401AF5
:10716000C008042101EB004004A101F085FE0020CD
:1071700010BD000088DB070038DB0700696E207750
:1071800065616B206E72665F6466755F696E6974B7
:107190005F757365720000001FB58908002201AB9E
:1071A000009283E80700684618DF04B010BD0000B5
:1071B0001FB5044B0FCB8DE80F00684618DF04B0F5
:1071C00010BD0000A8C607004FF4805041040860BD
:1071D0000020704770B50E460178134C062901D087
:1071E000012901D1017C217021780125012911D0CB
:1071F000022913D00D480E49401AC008012101EBA5
:1072000000400CA101F038FE0020207005207070B5
:10721000284670BD3146FFF799FDF9E73146FFF783
:107220000BFE0546F4E700004C2B002050DB070066
:1072300038DB0700496E76616C6964206F626A65AD
:107240006374207479706520696E2072657175654C
:1072500073742E0010B5040011D00120FFF794FEC6
:1072600000280BD100F0EEFC00F0CEFD48B109493A
:10727000081F00F057FD012803D0032010BD072090
:1072800010BD04480838C4600020FEF7AFF80020A5
:1072900010BD0000542B002010B5816889B10A4A46
:1072A0001821FCF7D7FC040009D008480849401A07
:1072B000C008022101EB004006A101F0DDFD2046DF
:1072C00010BD072010BD0000F172070050DB070061
:1072D00038DB07005363686564756C657220726102
:1072E0006E206F7574206F66207370616365210076
:1072F000AFF3008070B50546806886B020B9284994
:1073000040F2CF20FCF7BCFD182226496846FBF767
:1073100089F828788DF800002348244B2A78181A19
:107320000421C008224E01EB00440D2A1CD2DFE8E4
:1073300002F01B140714141B141B141B1B1B0C0042
:1073400020461CA101F098FD17E0204622A101F083
:1073500093FDF168072088470FE069462846FFF74C
:1073600039FF50B906B070BD032101EB004020A1E8
:1073700001F086FD02208DF801009DF801202046D5
:1073800023A101F07DFDD5E90112684690479DF8E3
:1073900001000128E6D0F16805208847E2E70000F7
:1073A000DCCD0700D0C6070038DB070050DB070044
:1073B0004C2B002048616E646C65204E52465F4441
:1073C00046555F4F505F524543454950545F4E4FBD
:1073D0005449465F5345540048616E646C65204EC5
:1073E00052465F4446555F4F505F41424F525400F2
:1073F000496E76616C6964206F70636F646520729A
:10740000656365697665643A20307825782E0000DA
:10741000526571756573742068616E646C696E671E
:1074200020636F6D706C6574652E20526573756C8A
:10743000743A20307825780038B105490160054953
:10744000416001210172002070470E20704700004A
:10745000597407009174070010B50C0001464FF0F5
:10746000110007D02278052A05D2DFE802F00F05C7
:107470000D0F0F000E2010BD084600F073F8002815
:10748000F9D10221217010BD112010BD082010BDBE
:107490000246082041B10B78022B04D1022A05D004
:1074A000032A00D1112070470E20704700200322CC
:1074B0000A70704770B510480024D0F82413491C96
:1074C00003D1D0F86403401C13D00C480C49401A77
:1074D000C008042101EB00400AA101F0CDFC4FF4EB
:1074E000FE25284601F0AAFEC9220349284601F0DC
:1074F000D5FE204670BD0000C047002060DB0700BD
:1075000038DB070045726173696E672073657474B8
:10751000696E67732070616765206164646974696E
:107520006F6E616C20646174612E000010B528B12B
:107530001C220349FAF776FF002010BD0E2010BD73
:1075400064F3070010B5064C00221821201DFDF73A
:1075500031FC2168814201D1012010BD002010BD05
:1075600064F3070070B50C4D0400D5F8640305F50D
:10757000597503D0401C03D0082070BD0E2070BD8B
:1075800000221821201DFDF715FC2060072221464E
:10759000284629DF70BD000000F00700014903F014
:1075A000F5BF000000F0070070B50546124813490A
:1075B000401AC408042000EB044011A101F05CFC57
:1075C0002846FFF7E1FC02004FF0010000EB044405
:1075D00002D0204613A108E000F06CF8002000F073
:1075E00051F9020005D0204619A101F049FC032001
:1075F00070BD002070BD000058DB070038DB0700BD
:1076000043616C6C696E67206E72665F6466755F5D
:1076100073657474696E67735F696E697428292E67
:107620002E2E00006E72665F6466755F666C617315
:10763000685F696E69742829206661696C656420D9
:1076400077697468206572726F723A20257800003D
:107650006E72665F6466755F73657474696E677376
:107660005F77726974655F616E645F6261636B7599
:10767000702829206661696C6564207769746820C8
:107680006572726F723A20257800000010B5FF22F3
:107690004FF400710648FAF7D7FE05482021243838
:1076A000FAF7D9FE024900205C39086310BD0000DA
:1076B0001C4800202DE9F05F4048FDF799FB404E43
:1076C000074634682046FDF793FB4FF0000A58B197
:1076D0006068012806D02046FDF79AF9D4F85C12BC
:1076E000884201D1012400E0002436483649DFF801
:1076F000DC80401AC00803214FF002094FF4607B80
:1077000001EB0045F7B1042101EB0040074630A131
:1077100001F0B2FB5A4629494046FAF783FEDCB134
:10772000384631A101F0A8FB366844465422311D89
:10773000201DFAF777FE4FF4327206F15C0104F176
:107740005C0007E06CB32846324901F095FB5A46CD
:107750001E483168FAF766FED8F80400444601284E
:107760001DD128462CA101F087FB3649402201F5A6
:10777000E470FAF757FE33491C22403101F5E470FA
:10778000FAF750FE84F860A2012184F8A1122E4875
:1077900084F8E2A2E169C0F82210C4F80490BDE8C0
:1077A000F09F4C4609EB0040284901F065FB594623
:1077B0000648FAF750FEC8F80440F0E700F007006A
:1077C0005C2B002058DB070038DB0700C047002097
:1077D0005573696E672073657474696E6773207082
:1077E0006167652E00000000436F7079696E672045
:1077F000666F7262696464656E2070617274732072
:1078000066726F6D206261636B7570207061676571
:107810002E0000008CCE07004F6C642073657474DA
:10782000696E677320706167652064657465637451
:1078300065642E20557067726164696E6720696E99
:10784000666F2E001C490020404A002028CE070009
:1078500070B50546094803F005FF084C2060204636
:10786000FDF7D6F8C4F85C02A4F5E0632A46214689
:10787000BDE87040024803F0FBBE0000C047002096
:1078800000F0070070B505460020FFF7E1FF040097
:1078900003D10349284603F079FE204670BD00005D
:1078A000C04700204FF48050704700002DE9F0479A
:1078B0001449DFF854808146A1EB0800C70813483B
:1078C00013490026401AC108042000EB0140054678
:1078D0003A4610A101F0D4FA00240EE008EBC400EF
:1078E000416848468847060006D028463346224667
:1078F00012A101F0CCFA02E0641CBC42EED3304687
:10790000BDE8F08728DB070020DB070088DB0700E5
:1079100038DB07005368757474696E6720646F778D
:107920006E207472616E73706F7274732028666F4C
:10793000756E643A20256429000000004661696C78
:10794000656420746F2073687574646F776E20743B
:1079500072616E73706F72742025642C2065727270
:107960006F722025640000002DE9F0471449DFF80C
:1079700054808146A1EB0800C7081348134900262C
:10798000401AC108042000EB014005463A4610A108
:1079900001F076FA00240DE058F834104846884784
:1079A000060006D028463346224612A101F06FFA9F
:1079B00002E0641CBC42EFD33046BDE8F087000013
:1079C00028DB070020DB070088DB070038DB070027
:1079D000496E697469616C697A696E672074726155
:1079E0006E73706F7274732028666F756E643A20C0
:1079F000256429004661696C656420746F20696E96
:107A0000697469616C697A65207472616E73706FF4
:107A100072742025642C206572726F7220256400B8
:107A2000012203F069B9000038B5144602780B460C
:107A3000FAB1012A09D0022A1DD0032A23D01749FE
:107A400040F2D930FCF71CFA25E0D0F801500022B2
:107A500021461846FDF7AEF9A8420AD01048114950
:107A60000122401AC008042101EB00400EA101F0E0
:107A700007FA012038BD01B02246BDE8304000239E
:107A8000401C00F023B8411C40220020009400F06C
:107A900017FA0128EED0002038BD0000BCD1070045
:107AA00068DB070038DB07004352432063686563E7
:107AB0006B206F6620617070206661696C65642E52
:107AC0002052657475726E20256400002DE9F04324
:107AD000A9B007462020894628901C4690460125DB
:107AE000782102A8FAF7B7FCFDF792F92CB1202211
:107AF000394620A8FEF7E6FE20AF24482449434635
:107B0000401AC608042000EB064004464A4621A15C
:107B100001F0BDF928A92C48CDE9000143464A46A9
:107B20002A4902A8FEF70EFE020006D0012000EB53
:107B3000064027A101F0A4F922E02022394622487C
:107B4000FAF79BFCE8B1022000EB06402DA101F002
:107B500093F9204632A101F08FF9204620223946C0
:107B600001F034F9204633A101F086F920462022A5
:107B7000154901F02BF900BF01F00EF80028FBD1E8
:107B8000002529B02846BDE8F083000068DB070027
:107B900038DB07004861736820766572696669633F
:107BA0006174696F6E2E20737461727420616464F5
:107BB000726573733A20307825782C2073697A6562
:107BC0003A20307825780000144F0020B8C3070011
:107BD000436F756C64206E6F742072756E206861DF
:107BE000736820766572696669636174696F6E2077
:107BF000286572725F636F64652030782578292E5E
:107C000000000000486173682076657269666963E8
:107C10006174696F6E206661696C65642E00000096
:107C200045787065637465642046572068617368A1
:107C30003A00000041637475616C2046572068610A
:107C400073683A0010B50648064C806B20B104F00A
:107C500031F808B1012000E00020207010BD0000C4
:107C6000C0470020602B00202DE9F041144C07464E
:107C70000D46E06BA26B0126411991420BD91148C8
:107C80001149401AC008012101EB00400FA101F089
:107C9000F3F8032610E00A492A465C3108443946C5
:107CA000FAF7C0FBE06B064A2844E06340322946FD
:107CB0003846FDF77FF820643046BDE8F0810000CB
:107CC000C047002068DB070038DB0700496E697495
:107CD00020636F6D6D616E64206C617267657220E8
:107CE0007468616E2065787065637465642E000049
:107CF00070B504004FF0010504D0B4F5007F03D93E
:107D0000042508E0032506E0044900200870FFF779
:107D1000BDFC03488463284670BD0000602B002032
:107D2000C04700202DE9F041064624480F46254B68
:107D3000D0E90E1222484FF00108C01AC00808EB23
:107D400000448A4205D020461FA101F095F808247E
:107D500030E0244D287840B1FEF736FE30603946D9
:107D6000E86804F0F9F9044624E003F0A3FFE0B169
:107D700000F050F80446002030603860012C0ED12D
:107D80003946E86804F0E8F90446012807D132468C
:107D90003968E86804F09CF90446012802D0FFF72E
:107DA00075FC07E085F8008004E020460EA101F094
:107DB00063F805242046BDE8F0810000C04700209C
:107DC00068DB070038DB070045786563757465205C
:107DD00077697468206661756C7479206F66667364
:107DE00065740000602B00204661696C6564207436
:107DF0006F206465636F646520696E6974207061CB
:107E0000636B657400000000014800787047000053
:107E1000602B0020F8B51C4C251D002094F86C3117
:107E2000014602463BB194F8D802B4F8DA2204F5D0
:107E3000B87504F53771154CA3680093636800F0BA
:107E40003FF80646012805D1281D00F043F90646F3
:107E5000012816D00E480F49401AC508022000EB31
:107E600005400DA101F008F8042000EB054510A124
:107E7000284601F001F82089616882B2284600F0A6
:107E8000A5FF3046F8BD0000404B0020602B0020CD
:107E900068DB070038DB070050726576616C696447
:107EA0006174696F6E206661696C65642E00000004
:107EB000496E697420636F6D6D616E643A000000F5
:107EC0002DE9F047A2B080462020DDF8A8900F46AB
:107ED00020909A461646782102A8FAF7BCFA0020AC
:107EE0002190FCF795FF40484049401AC5080320FF
:107EF00000EB054004463EA100F0BEFF57B1B8F1CB
:107F0000000F20460ED044A100F0B6FF162022B08C
:107F1000BDE8F087022000EB054045A100F0ACFF72
:107F20001320F4E74A4647A100F0AAFF20A94C48D5
:107F3000CDE900014B4652464A4902A8FEF702FC31
:107F400008B9402E01D00A20E1E7454832463946BB
:107F50004038FAF767FA204643A100F08DFF404809
:107F600020214038FEF77FFC3D4840214038CDE9D4
:107F70000001A0F148013A4A21A8209BFEF7BCFB72
:107F800002002BD0012000EB05403CA100F078FF5F
:107F9000042000EB054442A1204600F06DFF30496B
:107FA00020464022403900F011FF20463FA100F05A
:107FB00063FF20982A4982B2204600F007FF20463E
:107FC0003CA100F059FF204640223D4900F0FEFE52
:107FD00000F0E2FD0028FBD1052098E7204639A1FA
:107FE00000F04AFF012092E768DB070038DB07005A
:107FF0005369676E61747572652072657175697217
:1080000065642E20436865636B696E6720736967DA
:108010006E61747572652E00496E76616C696420BC
:108020007369676E6174757265207479706500009C
:108030004E6F207369676E617475726520666F7527
:108040006E642E0043616C63756C6174696E6720A9
:108050006861736820286C656E3A202564290000E9
:10806000F44E0020B8C30700566572696679207324
:1080700069676E6174757265000000005369676E10
:108080006174757265206661696C6564202865722B
:10809000725F636F64653A203078257829000000AC
:1080A0005369676E61747572653A00004861736860
:1080B0003A0000005075626C6963204B65793A00A4
:1080C00060C30700496D61676520766572696669FE
:1080D000656400002DE9F04104004FF0010603D172
:1080E0003349C420FBF7CCFE3248334A94F854108D
:1080F000801AC008012202EB004541B194F85500F6
:1081000040B1012806D0022804D0032802D0284616
:108110002AA147E01CB92649A320FBF7B1FE94F839
:108120006E00032805D028462AA100F0A5FE1426DB
:108130003BE094F8920018B194F89300002834D1F1
:10814000207A78B11C4A1B4B02209A1AD208E168A7
:1081500000EB0247342908D0384623A100F08CFEFA
:10816000112622E0284625A11CE0204603F074F9E0
:1081700030B1207880B12046FDF760F930B114E0CD
:10818000384622A100F078FE12260EE0384623A1E0
:1081900000F072FE102608E094F85500012804D083
:1081A000284623A100F068FE0F263046BDE8F08186
:1081B00004D2070070DB070038DB0700496E7661E8
:1081C0006C6964206669726D77617265207479707C
:1081D000652E0000496E76616C6964206861736881
:1081E00020747970652E00004661756C74792048A2
:1081F000572076657273696F6E2E00004E6F2048AF
:10820000572076657273696F6E2E0000534420729A
:108210006571206E6F74206D65742E004657207650
:10822000657273696F6E20746F6F206C6F772E00AC
:1082300046572076657273696F6E206D6973736936
:108240006E672E000FB438B5040003D110A1422090
:10825000FBF716FE606918B90DA14320FBF710FE6D
:10826000206818B90AA14420FBF70AFE606818B913
:1082700007A14520FBF704FE0599002905D006A8B3
:1082800000906A46204600F045F838BC5DF814FBC3
:108290002E2E5C2E2E5C2E2E5C2E2E5C2E2E5C65E1
:1082A000787465726E616C5C667072696E74665C1F
:1082B0006E72665F667072696E74662E630000008F
:1082C00010B5040003D107A13120FBF7D9FDA26846
:1082D000002A05D0D4E90403216898470020A06053
:1082E00010BD00002E2E5C2E2E5C2E2E5C2E2E5CE1
:1082F0002E2E5C65787465726E616C5C6670726956
:108300006E74665C6E72665F667072696E74662EFD
:10831000630000002DE9FC4791460C465FEA000827
:1083200004D183A140F25220FBF7AAFDD8F8140033
:1083300020B97FA14FF41570FBF7A2FDD8F800001B
:1083400020B97BA140F25520FBF79AFDD8F8040034
:1083500020B977A140F25620FBF792FD002C76D091
:1083600014F8011B39B125290ED04046FCF7ECFC6E
:1083700020780028F4D198F80C00002867D04046F7
:10838000BDE8FC47FFF79CBF0020012221782B2984
:108390001BD02D2902D0302908D102E040F0010085
:1083A00001E040F00200641C002AEFD100252A29D8
:1083B0000ED02178A1F130020A2A11D205EB8502F4
:1083C00001EB4205641C303DF1E740F00400EAE7B0
:1083D000D9F800100B1DC9F800300968641C0D4461
:1083E000217800232E290BD114F8011FA1F13002AE
:1083F0000A2A05D203EB830201EB4203303BF3E789
:108400006C290DD068290BD0692921D00BDC2529D6
:1084100018D0582931D063290ED0642915D117E01E
:1084200014F8011FECE7702969D0732932D075293F
:108430001BD0782909D120E0D9F80000011DC9F826
:10844000001001784046FCF77FFC641C90E76CE06C
:10845000D9F800100A1DC9F800200968CDE90050BC
:108460000A224046FDF774F9EFE7D9F800100A1D1B
:10847000C9F8002009680A2206E0D9F800100A1D90
:10848000C9F8002009681022CDE90050404603F0E9
:10849000C5FDDAE7D9F8001000270A1DC9F8002049
:1084A0000E68C00705D112E04046761C7F1CFCF721
:1084B0004BFC31780029F7D104E0202140466D1EA5
:1084C000FCF742FCBD42C0D9002DF6D1BDE74EB14C
:1084D0003046F9F7CBFF074604E0202140466D1EE9
:1084E000FCF732FCBD4206D9002DF6D103E0404630
:1084F000761CFCF729FC31780029F8D1A5E7D9F8DA
:108500000000011DC9F80010056830214046FCF745
:108510001BFC78214046FCF717FC08200021CDE920
:108520000001034610222946B0E7BDE8FC870000A1
:108530002E2E5C2E2E5C2E2E5C2E2E5C2E2E5C653E
:10854000787465726E616C5C667072696E74665C7C
:108550006E72665F667072696E74665F666F726D6A
:1085600061742E63000000002DE9F0411E4615469F
:108570000F46040003D11DA19E20FBF781FC20685B
:1085800018B91AA19F20FBF77BFC1DB917A1A020E9
:10859000FBF776FC39462046FBF770F940B93946BF
:1085A0002046FBF76BF918B910A1A320FBF768FC74
:1085B00060683946026820466A43FBF768F958B993
:1085C00060683946026820466A43FBF760F918B9CB
:1085D00006A1A520FBF754FC206833462A46D0F8B4
:1085E00010C039462046BDE8F04160472E2E5C2E73
:1085F0002E5C2E2E5C2E2E5C2E2E5C636F6D706FAB
:108600006E656E74735C6C69627261726965735CCD
:108610006673746F726167655C6E72665F667374B1
:108620006F726167652E630070B516460C460500D3
:1086300003D108A15520FBF723FC1CB905A1562046
:10864000FBF71EFC2C60314628462268BDE87040CE
:10865000104700002E2E5C2E2E5C2E2E5C2E2E5CE3
:108660002E2E5C636F6D706F6E656E74735C6C69DB
:10867000627261726965735C6673746F726167655B
:108680005C6E72665F6673746F726167652E6300FD
:108690002DE9F04128B1016819B1C969BDE8F0417F
:1086A00008470D4D0D480024461B14270DE000BF60
:1086B00004EB840005EB8000016829B1C969884793
:1086C00010B10120BDE8F081641CB6FBF7F0A042B8
:1086D000EED80020F6E70000F42B0020082C002044
:1086E000044801214174007A08B10020704701203C
:1086F000704700002C510020012801D0032808D128
:108700000449002201284A7400D00020087402F0B5
:1087100099BC70472C51002070B50146022801D049
:10872000032943D1224C207A00283FD0012831D0A0
:1087300002282FD11F4800230229006802D00329F4
:1087400028D119E0E360027912B1012A22D10BE0AD
:10875000D0E90565721B142A00D314222A448261D1
:108760004569AA420ED015E00169491C01614269C0
:1087700091420FD1237213E0E268521CE260082A92
:1087800008D9E360237202290AD00D21FCF7F5FD18
:1087900002F04EFC607C28B1BDE8704000F0A6BF3E
:1087A0000021F3E7BDE8704002F04CBC70BD000052
:1087B0002C510020842B00202DE9F8431D46089FF2
:1087C00016468846040003D12AA18820FBF758FBEF
:1087D0001EB928A18920FBF753FB206818B925A1F1
:1087E0008A20FBF74DFB1DB922A18B20FBF748FB2C
:1087F00060684068B5FBF0F100FB115141B1B5FB79
:10880000F0F100FB115018B11AA18E20FBF738FBD4
:108810004046FBF72DF838B94046FBF729F818B960
:1088200014A19120FBF72CFB3046FBF721F838B957
:108830003046FBF71DF818B90EA19220FBF720FB7C
:108840002A4641462046FBF722F848B92A464146C7
:108850002046FBF71CF818B906A19320FBF710FB84
:10886000009720682B463246C76841462046B847E5
:10887000BDE8F8832E2E5C2E2E5C2E2E5C2E2E5CF8
:108880002E2E5C636F6D706F6E656E74735C6C69B9
:10889000627261726965735C6673746F7261676539
:1088A0005C6E72665F6673746F726167652E6300DB
:1088B0002DE9FF411C46DDE90A7815460E4668465B
:1088C00000F010F846EA450141EA840141EA072236
:1088D00042EA0841009A00EB8200C0F80017BDE8A8
:1088E000FF81000010B5016804464A094FF00000FE
:1088F00002D0012A05D102E04FF0FF3001E040F242
:10890000FF3001F01F0201219140014204D108A172
:108910004FF4F670FBF7B4FA2068202802D24FF02B
:10892000A04010BD00F01F0020600C4810BD0000EA
:108930002E2E5C2E2E5C2E2E5C2E2E5C2E2E5C6D32
:108940006F64756C65735C6E7266785C68616C5C94
:108950006E72665F6770696F2E68000000030050DA
:1089600010B5016804464A094FF0000002D0012A00
:1089700005D102E04FF0FF3001E040F2FF3001F09E
:108980001F0201219140014204D108A14FF4F67069
:10899000FBF776FA2068202802D24FF0A04010BDE5
:1089A00000F01F0020600C4810BD00002E2E5C2E31
:1089B0002E5C2E2E5C2E2E5C2E2E5C6D6F64756CE4
:1089C00065735C6E7266785C68616C5C6E72665F23
:1089D0006770696F2E6800000003005038B50124ED
:1089E0000090684631B1FFF77DFF00998C40C0F8D8
:1089F000084538BDFFF776FF00998C40C0F80C455C
:108A000038BD000030B5134B014600201C692246DA
:108A10000AE0D2681579854205D1401C0A28F6DBA8
:108A20004FF0FF3030BD1268002AF2D1421CF9D05D
:108A3000CA6810711A693AB1D268CC6812682260AB
:108A40001A69D268116030BD1961C96800220A60D4
:108A500030BD0000D86200207047FAF751BD704762
:108A600008B5034A00924023024A00F005F808BD09
:108A70003DB5070040510020F0B595B01C461546A5
:108A80000E4608461A9F00F069FB182109A8F9F75D
:108A9000E2FC0E97CDE909540023082203A93046D1
:108AA00000F072FB05980690BDF81000ADF81C00B0
:108AB000BDF81200ADF81E0000208DF821000399CA
:108AC000082501F00300012802D0022816D02FE06B
:108AD000C1F3C200C1F383178C0A8DF82000BA00DD
:108AE0002B460FA9304600F04FFB09A8009006ABBB
:108AF0003A460FA9204600F08DFA19E0C1F3C200F2
:108B00008C0D8DF82000082C01D2274600E00827A4
:108B10002B463A460FA9304600F036FB3D44E41B95
:108B200009AB06AA39460FA800F0DAF9002CEAD101
:108B3000304600F019FB15B0F0BD00000A4A0129CB
:108B400002EBC00007D0022907D0032907D004296F
:108B500007D000207047022070470420704700793A
:108B6000704740797047000038DB070010B5FFF709
:108B700074FF04210648FFF745FF002803DA054982
:108B80004120FBF77DF902490120C968487110BDF9
:108B900028DB070090D607002DE9F04F8DB0FCF7D9
:108BA000EBF818B100200DB0BDE8F08F7C4E00202E
:108BB000B061BFF34F8FA6F580547A49A068029048
:108BC0000D684FF00009284004EB80000AE0B0690E
:108BD00070B961680298814201D8A160E2E728403B
:108BE00004EB80000C3002A9FCF705FE0028EED152
:108BF000002009AAA046029901EA050308EB8303B5
:108C0000491CDB6842F82030401C02910228F2D354
:108C1000099800F00301022902D001294CD0A6E0F6
:108C2000810D50228A46B2EB905F00D850210C464D
:108C300064F39F50099008315B4800F046FA070042
:108C400074D000F08BFA4B46082209A9384600F090
:108C5000C9FA029909F1080B2940681A8000001D21
:108C6000844222D9514D30B1C2B208EB8101201AA1
:108C700091460C3104E02946E2B20025914628468F
:108C8000C4B25B46384600F0ADFA0BEB09032DB1D8
:108C9000224629464FEA070000F0A4FA02990AF199
:108CA000030001EB9000029039E008EB81015B4684
:108CB000224638460C31EFE7C0F38311062900D372
:108CC000062161F389100990C0F38310801C810094
:108CD000354800F0FAF9070049D000F03FFA4B465A
:108CE000082209A9384600F07DFA09F10809002494
:108CF0000FE002984B4600EA0501401C08EB810199
:108D00000290042238460C3100F06CFA09F1040993
:108D1000641C0998C0F38310A042EAD837B13469C3
:108D2000B06978B1384600F01FFA34E01FE0E0681F
:108D30004079012804D122682046394612689047BC
:108D4000E0680468002CF2D1384600F00DFA0020EB
:108D50008DF800006846FBF703F8B06910B9029976
:108D6000C8F808109DF80000FBF746F813E03469D6
:108D700005E02168204689688847E0680468002C7F
:108D8000F7D10B480B49401AC008022101EB004003
:108D900009A100F071F8FBF7EFFF80F0010002E796
:108DA000D8620020982B0020BCDB0700E452002092
:108DB00088DB070038DB07004261636B656E647314
:108DC00020666C7573686564000000002DE9F84F3B
:108DD0008146274FD01C15468A46800800226946E6
:108DE0003E68FBF757FFDFF88C80B0B3009CA01CF7
:108DF000009039683040091A8F003F1DBD4208EBD2
:108E0000800002D82A46514608E03A4651460C30C6
:108E1000F9F708FB1748EA1B0AEB07010C30F9F7D2
:108E200001FB4FEA1947FCF739FA47EA0042601C98
:108E3000304008EB8000344008EB8401C260C86811
:108E40004FF6C07269F3C500904365F39F5020F060
:108E50000300801C20F00400C86098F8000001E0C6
:108E6000FFF79AFE0028FBD1FCF771FDBDE8F88FF3
:108E7000982B0020D852002000231A4602F0E4BEAE
:108E800008B5012300926A4602F0DEFE08BD1CB55B
:108E9000CDE9002302236A4602F0D6FE1CBD3EB592
:108EA000069C8DE81C0003236A4602F0CDFE3EBD01
:108EB0007FB5DDE908458DE83C0004236A4602F0F1
:108EC000C3FE7FBD70B586B00DF1280C9CE8700024
:108ED0008DE87C0005236A4602F0B6FE06B070BD40
:108EE0002DE9F0470E4680461C469246082940D898
:108EF00094F80C90002020731946104602F03EF8BA
:108F00000025B54206D218F805201BA12046FFF720
:108F100099F903E01AA12046FFF794F96D1C082D7A
:108F2000EFD318A12046FFF78DF90025B54212D2E4
:108F300018F805707E2F08D8F9F770FA0068C05D40
:108F400010F03E0F01D03A4600E02E220EA120463E
:108F5000FFF778F903E00DA12046FFF773F96D1CC8
:108F6000082DE3D301222146504601F0A7FE84F8E4
:108F70000C90BDE8F087000020253032780000001A
:108F8000202020007C00000025630000200000005D
:108F9000064910B500200870054800F0E3F80028E5
:108FA00003D1044800F09CF9002010BDD8520020E5
:108FB000BCDB0700A8C9070002480349401AC008E3
:108FC00070470000A8DB070038DB070013B56846D0
:108FD000FCF7FCFD08B100201CBD0248009950F8C8
:108FE00031001CBD38DB070070B509480125046954
:108FF000A0F58050057007E0E068457121682046C3
:1090000049688847E0680468002CF5D170BD00000D
:10901000D86200202DE9FF4781460C9D00200C46B8
:109020002F7B2873984616462946184601F0A6FF5E
:10903000072E42D2DFE806F004090F161F2A360079
:1090400049462846FFF7FEF837E049462846226899
:10905000FFF7F8F831E0D4E9002349462846FFF746
:10906000F1F82AE0A0680090D4E900234946284698
:10907000FFF7E8F821E0D4E90201CDE90001D4E9E5
:10908000002349462846FFF7DDF816E004F1080002
:1090900007C88DE80700D4E9002349462846FFF7B2
:1090A000D1F80AE004F108000FC88DE80F00D4E9F8
:1090B000002349462846FFF7C5F8002229464046C6
:1090C00001F0FCFD2F73BDE8FF872DE9F041058A13
:1090D00080462D1F4819C01CB0FBF5F0C6B24046B3
:1090E000FCF706FE041E19D00020207101206071DB
:1090F000E58000272546761EC4F800800BE0404638
:10910000FCF7F6FD60B16179491C61712860054684
:109110007F1CC0F80080B742F1D32046BDE8F08143
:10912000204600F002F80020F8E72DE9F0414579EB
:1091300001466B1E002201E00968521C9A42FBD3D3
:109140000F680146002605E038460C68FCF736FE3D
:109150002146761CAE42F7D3BDE8F0810121001D07
:10916000FCF79FBDFCF772BE10B504460121001D3F
:10917000FCF7B8FD10F0FF0F04D12046BDE8104009
:10918000FFF7D3BF10BD00001CB514460122CDE986
:10919000002401AAFCF7ACFC0198A04204D003A172
:1091A0004FF48070FAF76CFE1CBD00002E2E5C2E72
:1091B0002E5C2E2E5C2E2E5C2E2E5C636F6D706FDF
:1091C0006E656E74735C6C69627261726965735C02
:1091D0006D656D6F626A5C6E72665F6D656D6F6204
:1091E0006A2E63001CB514460022CDE9002401AAB2
:1091F000FCF77EFC0198A04203D002A1F620FAF70A
:109200003FFE1CBD2E2E5C2E2E5C2E2E5C2E2E5C68
:109210002E2E5C636F6D706F6E656E74735C6C691F
:10922000627261726965735C6D656D6F626A5C6EB6
:1092300072665F6D656D6F626A2E63000949022276
:109240000A60BFF36F8FBFF34F8F0A1D106006488F
:109250000268002AFCD000200860BFF36F8FBFF3C4
:109260004F8F704704E5014000E40140094A0123A3
:109270001360BFF36F8FBFF34F8F01600648016823
:109280000029FCD000201060BFF36F8FBFF34F8F19
:109290007047000004E5014000E4014070B50E4C49
:1092A00001232360BFF36F8FBFF34F8F00230B4D5C
:1092B00008E000BF51F8236040F823602E68002EBC
:1092C000FCD05B1C9342F5D300202060BFF36F8F6E
:1092D000BFF34F8F70BD000004E5014000E4014082
:1092E00082680021916082681161826851618268A0
:1092F000D1608268516080680160704708B50022C3
:1093000042504058009008BD20B1034909680160EF
:10931000002070470E2070472CCA07002DE9FE433D
:1093200007460E460846FFF7EFFF00287CD10024D1
:109330000094019406208DF800704FF00108ADF8FC
:10934000040002948DF8028069462020326869DFAB
:109350003649374A891AC908012202EB014530B162
:1093600000F09EFA024628463249FFF789FD009434
:109370008DF801808DF80240019402948DF803402D
:1093800069464020326869DF30B100F089FA024650
:1093900028462949FFF774FD00948DF80070F720E6
:1093A000ADF802000194029469462320326869DF17
:1093B00030B100F075FA024628462049FFF760FDFB
:1093C0000094019402948DF800806946012032686F
:1093D00069DF30B100F064FA024628461849FFF709
:1093E0004FFD4FF4B0600090019402946946A120B3
:1093F000326869DF30B100F053FA0246284611495D
:10940000FFF73EFD0094019402948DF800406946F8
:10941000A020326869DF30B100F042FA02462846E7
:109420000949FFF72DFD0020BDE8FE8398DB07000A
:1094300038DB070088D80700D0D807001CD9070000
:10944000E8D7070034D8070094D707002DE9F0418A
:109450000546076860DF804619491A482A68081AD5
:10946000C608BA4219D9022000EB064416A12046CC
:10947000FFF702FD20463A461FA12B68FFF707FDC4
:109480004FF08050D0F80C012968800200F10050A4
:10949000421A204625A1FFF7F3FCB8F100004FF077
:1094A00001040AD000F0FCF9024604EB06402AA1B0
:1094B000FFF7E6FC4046BDE8F0812F480470F9E76D
:1094C00098DB070038DB0700496E737566666963D1
:1094D00069656E742052414D20616C6C6F636174DC
:1094E000656420666F722074686520536F667444EB
:1094F00065766963652E00004368616E6765207458
:1095000068652052414D207374617274206C6F63E2
:109510006174696F6E2066726F6D203078257820D7
:10952000746F20307825782E000000004D61786936
:109530006D756D2052414D2073697A6520666F729A
:10954000206170706C69636174696F6E206973204B
:10955000307825782E00000073645F626C655F656B
:109560006E61626C6528292072657475726E65641F
:109570002025732E00000000EF2B002030B5184886
:10958000ADF5017D0078002826D04FF4FA7400BFB5
:10959000ADF8004280A9684661DF38B105281BD0CC
:1095A0000DF5017DBDE83040FAF798BA6D460D49DA
:1095B0007DA800F0F1F809E07DA800F0D5F8D0E929
:1095C0000021284690477DA800F024F97DA800F0EE
:1095D000CBF80028DCD0EFE70DF5017D30BD0000B1
:1095E000EF2B002030CA0700F8B5134C2078C0B12B
:1095F0000120A07001F06CFF112814D0022001F0AE
:1096000083FF00258DF800506846FAF7A9FB11DFAB
:10961000064625709DF80000FAF7EEFB2EB13046A5
:10962000F8BD0820F8BD0020F8BDA57002F02CFAA6
:10963000032001F069FFF6E7EC2B00207CB5194C04
:10964000207808B108207CBD0120A070002001F026
:109650003FFF112819D0002001F056FF12480026C4
:10966000006801908DF800606846FAF779FB0F49B1
:1096700001A810DF05000AD0002020709DF800002E
:10968000FAF7BAFB2DB128467CBD00207CBD012035
:10969000F3E7A670667002F05BFA012001F034FF78
:1096A000F3E70000EC2B0020C4C90700793A07005B
:1096B0000EB50A49684600F06FF808E0684600F009
:1096C00047F8D0E900108847684600F0A3F86846DC
:1096D00000F03EF80028F1D10EBD0000E0C90700FF
:1096E0000148007870470000EC2B00200548817885
:1096F00019B1007818B1FFF777BF08207047FFF75E
:109700009DBF0000EC2B00201FB568464BDF30B139
:10971000052819D004B0BDE81040FAF7DFB90B49AD
:1097200001A800F039F809E001A800F029F8D0E913
:1097300000210098904701A800F06CF801A800F003
:109740001FF80028E1D0EFE71FBD00004CCA07005A
:1097500010B5040003D10349C420FAF791FBA068B7
:1097600010BD000040D7070010B5040003D1034925
:10977000C420FAF785FBA06810BD000040D70700A1
:1097800010B5040003D10349C420FAF779FBA0689F
:1097900010BD000040D7070070B50D46040003D18E
:1097A00008495020FAF76CFB1DB906495120FAF719
:1097B00067FB2560286860602046BDE8704000F0C7
:1097C00003B8000050D2070010B5040003D11049BF
:1097D0003320FAF755FB206818B90D493420FAF701
:1097E0004FFB606818B90A493520FAF749FBD4E9FC
:1097F00000104A68904201D1002004E0D0E9002323
:109800009A4202D01046A06010BD08306060F0E7B8
:1098100050D2070010B5040003D112496320FAF7B3
:109820002FFB206818B90F496420FAF729FBA068BC
:10983000002815D0216889680844A060606818B9BC
:1098400008497320FAF71CFBD4E9010142689142F0
:1098500006D1083060602046BDE81040FFF7B4BF75
:1098600010BD000050D207000C4A10B502F59473E9
:109870000EE0991AC91001EBD171491002EBC10138
:109880000C68844201D90B4602E005D201F10802BE
:109890009A42EED3002010BD486810BD68C707008B
:1098A00000B5FFF7E1FF002800D1014800BD00002E
:1098B00054C707002DE9F04104461348134BC01A62
:1098C0000C21B0FBF1F6A0694FF0FF3110F8022C2B
:1098D00002B92169002011E000EB400503EB85058A
:1098E0002F68974209D14F1C02D06F688F4204D174
:1098F00094E80F00AD68A84703E0401CB042EBD3EA
:1099000001202060BDE8F0810CDC070000DC0700CE
:1099100010B5144612680830202A02D248F21450BA
:1099200010BD002201F03CFF0028F9D1202020606A
:10993000002010BD083001F0BBBF083002F07AB83B
:1099400002480068002800D0012070470004014050
:1099500003490860034801680029FCD070470000F3
:1099600004E5014000E4014070B50C46050004D157
:109970000F494FF48270FAF783FA24B90C4940F288
:109980000510FAF77DFA0B480B49401AC00804216C
:1099900001EB004009A1FFF76FFA13490320C968E2
:1099A00088476869FEF7A4F9FBF711FD607070BD88
:1099B000DCCD070050DB070038DB070048616E6430
:1099C0006C65204E52465F4446555F4F505F4F4294
:1099D0004A4543545F4352454154452028636F6DC7
:1099E0006D616E64290000004C2B002070B50D469F
:1099F00020B916494FF49670FAF742FA25B913497F
:109A000040F22D10FAF73CFA11481249401AC108E9
:109A1000042000EB014004460FA1FFF72DFA19497D
:109A2000081FFEF77FF9FBF7D2FC6870012805D10B
:109A30000020FDF727FF10B10A20687070BD204696
:109A4000BDE8704010A1FFF717BA0000DCCD070099
:109A500050DB070038DB070048616E646C65204E00
:109A600052465F4446555F4F505F4F424A4543540C
:109A70005F455845435554452028636F6D6D616EB1
:109A800064290000542B002057726974696E6720A6
:109A900076616C696420696E697420636F6D6D61B5
:109AA0006E6420746F20666C6173682E0000000085
:109AB00070B50D46040004D11A494FF48970FAF7C5
:109AC000DFF9206920B9174940F21310FAF7D8F9E5
:109AD000A08A20B913494FF48A70FAF7D1F925B951
:109AE000104940F21510FAF7CBF90F480F49401A08
:109AF000C008042101EB00400DA1FFF7BDF9A18AC8
:109B00002069FEF7B1F8FBF762FC68702846FBF7A6
:109B10003FF9E168002903D02069BDE8704008479B
:109B200070BD0000DCCD070050DB070038DB07000C
:109B300048616E646C65204E52465F4446555F4FE7
:109B4000505F4F424A4543545F575249544520287D
:109B5000636F6D6D616E64290000000030B587B0E1
:109B60000C46054618221C496846F8F75BFC207B2A
:109B700001951A4D8DF80000012806D0022817D053
:109B8000062823D1607B049020E0A888E880607BD1
:109B90000490217CE08961F31F40617C40EA016010
:109BA00005900498012811D10D48FDF77FFE0DE0C6
:109BB0000C480D49401AC008042101EB00400BA1DC
:109BC000FFF75AF9B4F80D00A880E8806846FDF761
:109BD00063FB07B030BD0000F8C507002C2B002048
:109BE00020DB070040DB070038DB070053657420EB
:109BF00072656365697074206E6F74696600000039
:109C000070B50E460B480C49401AC108042000EB01
:109C100001440AA12046FFF72FF9114D204611A15A
:109C2000AB6C2A6DFFF733F9A86CB060286D7060DB
:109C300070BD000050DB070038DB070048616E6430
:109C40006C65204E52465F4446555F4F505F43520D
:109C5000435F474554202864617461290000000077
:109C6000C04700204F66667365743A25642C204314
:109C700052433A3078253038780000002DE9F84F0B
:109C80000D460746374838494FF00409401AC408C2
:109C900009EB0440064635A1FFF7EEF8FEF7B4F8ED
:109CA000012101EB04444FF0080AA8B17A694FF092
:109CB0000308B2B137493848130515D0436DD1F8C0
:109CC00008C0134463450FD0204634A1FFF7D4F8F1
:109CD00085F80180BDE8F88F204639A1FFF7CCF860
:109CE00019E0204644A1F1E7B2F5805F06D920468D
:109CF00048A1FFF7C1F885F80190EBE7436DD1F873
:109D000008C003EB0208E04508D920464A49CDF8CF
:109D100000C0FFF7C4F885F801A0DBE74264C26C1D
:109D200003650363804682647869002200F6FF7051
:109D3000070B486839461844FDF7BCF830B1204697
:109D40003EA1FFF799F805206870C3E7D8F84810DE
:109D5000009130463FA1D8F85030D8F84420FFF7A2
:109D60009EF8B7E750DB070038DB070048616E64F8
:109D70006C65204E52465F4446555F4F505F4F42E0
:109D80004A4543545F435245415445202864617419
:109D9000612900004C2B0020C04700204F626A65FB
:109DA00063742073697A65206D7573742062652011
:109DB0007061676520616C69676E65640000000012
:109DC00043616E6E6F7420637265617465206461B7
:109DD0007461206F626A65637420776974686F7557
:109DE000742076616C696420696E697420636F6D9C
:109DF0006D616E64000000004F626A6563742073D9
:109E0000697A652063616E6E6F7420626520302E02
:109E100000000000496E76616C69642073697A65A0
:109E200020666F72206F626A6563742028746F6F9A
:109E3000206C61726765290068CD07004572617307
:109E400065206F7065726174696F6E206661696C00
:109E5000656400004372656174696E67206F626AB1
:109E600065637420776974682073697A653A202580
:109E7000642E204F66667365743A2030782530383A
:109E8000782C204352433A2030782530387800002F
:109E90002DE9F0410E46074615481649401AC508F7
:109EA000042000EB054014A1FEF7E6FF1C4CD4E9AA
:109EB0001401626C431A9A420AD0012000EB05405B
:109EC00018A1FEF7E4FF082070700120BDE8F081C2
:109ED00000216164A16CE16460650021384600F0F6
:109EE00035F819490420C96888470020EEE70000CA
:109EF00050DB070038DB070048616E646C65204E5C
:109F000052465F4446555F4F505F4F424A45435467
:109F10005F455845435554452028646174612900C4
:109F2000C0470020496E76616C6964206461746189
:109F30002E2065787065637465643A2025642C2052
:109F4000676F743A202564004C2B0020F0B504465E
:109F500087B00020FEF79CFB01002548254A4FF002
:109F60000107A0EB02004FEAD0050AD0224A1821CF
:109F70002046F9F76FFE020037D007EB05401FA11E
:109F800031E0182228496846F8F74CFA2748284E4D
:109F9000184B174D016DEB1A0420DB08B26800EB7B
:109FA0000345914215D1284622A1FEF765FFD6E967
:109FB0000101FDF735FD8DF80100FBF708FA8DF87A
:109FC0000100D4E90112684690472648FDF75AFC83
:109FD00005E08DF80170D4E90112684690479DF8BC
:109FE0000120284620A1FEF74BFF07B0F0BD00007E
:109FF00050DB070038DB07004D9F07004661696CA6
:10A00000656420746F207363686564756C65206F88
:10A01000626A65637420657865637574653A20309B
:10A020007825782E00000000B8C60700C047002041
:10A030004C2B002057686F6C65206669726D7761E4
:10A04000726520696D616765207265636569766513
:10A05000642E20506F737476616C69646174696EEC
:10A06000672E000021A20700526571756573742088
:10A0700068616E646C696E6720636F6D706C657487
:10A08000652E20526573756C743A203078257800FF
:10A0900038B50D460C480D49401AC108042000EBA4
:10A0A000014004460AA1FEF7E7FE134813A1826CA3
:10A0B000AA60036D4FF480506B60E860009020460A
:10A0C000FEF7EDFE38BD000050DB070038DB07006F
:10A0D00048616E646C65204E52465F4446555F4F42
:10A0E000505F4F424A4543545F53454C45435420CB
:10A0F0002864617461290000C047002063726320F6
:10A100003D20307825782C206F6666736574203D7D
:10A1100020307825782C206D61785F73697A65200E
:10A120003D203078257800002DE9F0410E460446A8
:10A1300026482749401AC708042000EB074025A1FC
:10A14000FEF79AFEFDF760FE90B12C4DD5E91401A3
:10A15000401AA18A6A6C084490420BD9012000EB96
:10A16000074027A1FEF788FE03207070BDE8F0814C
:10A170000820FAE7284A286B526800EB02081F4AB9
:10A1800020694832FAF716FE0746E06820B92349ED
:10A190004FF4F870F9F774FED4E90331A28A40460F
:10A1A000FCF73EFF20B1D4E90310BDE8F0410847B9
:10A1B000A18A286B08442863A18A286DAF640844EB
:10A1C0002865B760286D7060D0E7000050DB07009D
:10A1D00038DB070048616E646C65204E52465F4470
:10A1E00046555F4F505F4F424A4543545F5752496F
:10A1F000544520286461746129000000C047002094
:10A200005772697465207265717565737420746F17
:10A210006F206C6F6E6700004C2B0020DCCD0700B8
:10A220000848094910B5401AC008042101EB004054
:10A2300006A1FEF721FE12490620C968BDE81040BC
:10A240000847000050DB070038DB0700416C6C203A
:10A25000666C617368206F7065726174696F6E738C
:10A26000206861766520636F6D706C657465642E1F
:10A270002044465520636F6D706C657465642E00D4
:10A280004C2B0020FEF7B0FEFEF786FC0028FBD129
:10A290000D4E64254FF47A47741C3846A0476D1E56
:10A2A000FAD10A480068C00700D000BEBFF34F8F44
:10A2B0000648E4380168064A01F4E0611143016090
:10A2C000BFF34F8F00BFFDE7A0C30700F0ED00E034
:10A2D0000400FA0510B50446084809492246401A08
:10A2E000C008042101EB004006A1FEF7C9FD21468C
:10A2F000BDE810400848FBF761BD000040DB0700E7
:10A3000038DB070046726565696E672062756666B0
:10A310006572202570000000A8DB070030B58A1D9B
:10A320008B79083187B0022B33D153888489A342BB
:10A330002FD1127A012A2CD1184C0DF1040C3CCCEF
:10A340008CE83C000A89ADF80C204A890C31049154
:10A350001249ADF80E208039114C096A0591CDF8EB
:10A3600018D0018A05AA6088ADDF18B96846FAF7E7
:10A37000D3FA38B10020ADF8080001A96088B0DF39
:10A3800050B106E040F2FD10ADF8080001A9608868
:10A39000B0DF002007B030BD0120FBE710C607008A
:10A3A0002C2B002070B506468C1DC888B18888B05B
:10A3B00088422DD11B48FBF79BFC05001A481B491E
:10A3C000A0EB01004FEAD00024D0F4210091042139
:10A3D00001EB004063892A4615A1FEF760FD628902
:10A3E00004F10C012846F8F71DF81822184901A8B5
:10A3F000F8F718F8029605956089ADF8180001A8DD
:10A40000FCF74AFF002803D029460648FBF7D6FC94
:10A4100008B070BD022101EB00400EA1FEF72CFD3B
:10A42000F6E70000A8DB070040DB070038DB070089
:10A430004275666665722025702061637175697268
:10A4400065642C206C656E20256420282564290015
:10A4500020C6070063616E6E6F7420616C6C6F6361
:10A46000617465206D656D6F7279206275666665D1
:10A4700072210000F8B50D4614460646694600F004
:10A480005DFA00280FD0009BB3F5803F0AD2981CDC
:10A49000834207D8A9780222B2EB911F02D0298902
:10A4A000814201D20020F8BD2380A11C3046009AD1
:10A4B00000F09AFBF8BD114600F0D5B8114600F047
:10A4C000E7B8F8B50C4615460646694600F036FA78
:10A4D00000280CD0009A501C904207D3A178022388
:10A4E000B3EB911F02D02189814201D20020F8BD37
:10A4F0002946304600F078FB009A0021A954F8BDA7
:10A500002DE9FF410C46CE6817460546694600F026
:10A510003DFB00280ED0E06800280BD0A0783A461A
:10A52000C0F3011002283146684606D000F0DEF87C
:10A530000199696004B0BDE8F08100F085F8F7E7A3
:10A540007CB50D461446694600F095F9002820D0E8
:10A550002889082806D0042809D002280AD0012812
:10A560000CD015E0DDE90001C4E900010AE0009823
:10A57000206006E0009800B2208002E0009840B21F
:10A580002070C117DDE9002350405940084301D035
:10A5900000207CBD01207CBD7CB50D46144669467B
:10A5A00000F0A7F9002820D02889082807D000212A
:10A5B000042809D002280AD001280CD014E0DDE9D3
:10A5C0000001C4E9000109E00098206006E000985D
:10A5D00080B2208002E00098C0B22070DDE9002344
:10A5E00050405940084301D000207CBD01207CBD73
:10A5F0007CB50D461446694600F07BF9002820D052
:10A600002889082808D00099CA1704280BD00228E6
:10A610000CD001280DD013E0DDE90012C4E90012CE
:10A620000846134608E00846216004E008B220808E
:10A6300001E048B22070C31748405340184301D08E
:10A6400000207CBD01207CBD70B50D460646144639
:10A650001146284600F0B5FA224629463046BDE8A4
:10A66000704000F043B838B50C460422694600F04B
:10A67000BBFA00280BD09DF80210BDF8000061F372
:10A680001F409DF8031040EA01602060012038BDA2
:10A690001CB50C460822694600F0A6FA002824D012
:10A6A0009DF801109DF800209DF80230080E42EA46
:10A6B000012242EA034240EA13409DF803309DF82C
:10A6C000041040EA132008439DF8051042EA036293
:10A6D00040EA01209DF8061040EA01409DF807106D
:10A6E00040EA0160C4E9002001201CBD2DE9F04FC3
:10A6F00005469DB000200F90064610904FF0FF3A9F
:10A7000001A800F07FF94FF0010B0DF13C0983E047
:10A7100012AB6A460BA9284600F0CAF850B101A84E
:10A72000009900F080F960B10298807810F0300F45
:10A7300054D061E09DF84800002871D11DB0BDE8FB
:10A74000F08F0098B04243D3029C01AE029880780B
:10A7500000F00F00082812D0304600F07BF9029874
:10A76000A042F3D156460098B04231D3D5F80880C4
:10A7700007909DF82C000E900598046821E002983F
:10A780000688F0E7206807682FB1214628460E9B0F
:10A79000079AB84712E01195216807980E9F8968BB
:10A7A000098881420CD1214617A8FBF7B9F884F833
:10A7B0000CB017AA39461198FAF795FB0028BDD0BE
:10A7C000A46814B1A9684145DCD0A968414523D1EA
:10A7D0009DF82C10284600F043FA1BE0039840280F
:10A7E0000AD200F01F000BFA00F20398400959F852
:10A7F0002030134349F82030EC682CB101AB9DF8B0
:10A800002C2028460099A04701AA9DF82C10284624
:10A81000FAF769FB002891D0A86800287FF478AF88
:10A82000DDE90204857801A800F014F90028F7D1C9
:10A8300015F0300F03D10298008800B1641CC4B138
:10A840000020494605E000BF51F82020521C0ED1DF
:10A85000401CB0EB541FF7D3600959F8201004F0E6
:10A860001F00C0F120022AFA02F0814201D000202C
:10A8700064E7012062E71CB50C46694600F039F830
:10A88000002814D0DDE90002C10709D051084FEAC1
:10A8900030006FEA00026FEA0100C4E9002004E022
:10A8A00051084FEA3000C4E900014FF001001CBD1F
:10A8B000F8B507460020187008700E4610601C4658
:10A8C00015466946384600F039F801004FF001009E
:10A8D00009D0009959B1C8082860009800F0070015
:10A8E00030700120F8BDB96809B10020F8BD2070B2
:10A8F000FBE72DE9F8430026884681463446354675
:10A9000004E0402E02D30020BDE8F88369464846A3
:10A9100000F096F90028F7D09DF80070324607F055
:10A920007F00C10FF7F76AFD29430443F61D0D466A
:10A930003806E6D4C8E900410120E5E7F8B50E463F
:10A940000746694600F07CF900280AD09DF80040CF
:10A95000200616D5072504F07F0403E0202D01D33F
:10A960000020F8BD6946384600F06AF90028F8D0A2
:10A970009DF8001001F07F00A8400443ED1D08067B
:10A98000ECD401203460F8BD30B45968114AC9686C
:10A99000914208D1D0E901120F48D0E90134234394
:10A9A00003D00021817030BC704711F8013BA2F147
:10A9B00001021B06F9D4C0E9011201218170074888
:10A9C000074930BC401AC008042101EB004005A132
:10A9D000FEF756BA40C40700602B002068DB070072
:10A9E00038DB070050423A20496E69742070616379
:10A9F0006B65742064617461206C656E3A20256417
:10AA000000000000C26000230160C0E901138B88D0
:10AA10001A440261B1F906301A44426108880028DC
:10AA200000D00120704770B545680E460446606846
:10AA30000188B14206D1807800F00F00082801D0CB
:10AA4000012070BD204600F005F86068A842EED1F4
:10AA5000002070BD30B541680A885AB101F1100379
:10AA600043600A8A42B18C780A89C4F30115032D28
:10AA700007D00BE0002030BDC2680168FFF7C2FFBD
:10AA8000F8E79D78C5F30115032D06D00225B5EB37
:10AA9000141F08D14C89624309E08D8804690022A3
:10AAA000641B046103E0B5EB941F00D10422897894
:10AAB00011F0300F02D18168491C81609C880169C6
:10AAC000214411440161B3F9062011444161012080
:10AAD00030BD30B54168002487B0897801F00F029D
:10AAE000082A11D08A091ED00222B2EB911F09D187
:10AAF0000269C1F301110229146001D0032901D1B7
:10AB00004069048007B030BD0069056808E02C7317
:10AB100029466846FAF704FF6846FFF7DAFFAD6892
:10AB2000002DF4D1EEE7C1F30111012912D0022961
:10AB3000E6D00329E4D04268917801F00F0107299B
:10AB40000BD0D16881B11289006907B0BDE83040EF
:10AB5000F7F768BC41690C70EDE70169D06807B090
:10AB6000BDE8304000F02DB81189006907B0BDE89C
:10AB70003040F7F770BC000010B5034B002408C04C
:10AB800080E8160010BD00002D4D070038B50D46B9
:10AB900004466946FFF7D2FE00280BD0D4E9000234
:10ABA000D4E90213C5E90002C5E902130098814205
:10ABB00001D2002038BDA860A168081AA060012059
:10ABC00038BD00B50A4687B001466846FFF71AFF50
:10ABD000002807D06846FFF77CFF6846FFF73AFF7A
:10ABE0000028F7D107B000BD7FB514460546A9B9C6
:10ABF000124A2868904208D110E01022694628467F
:10AC0000FFF7F2FF002807D0103C102CF5D82246A1
:10AC100069462846FFF7E8FF04B070BDA868A04267
:10AC200001D20020F8E72B682246284698470028E2
:10AC3000F2D0A868001BA8600120EDE72D4D0700A9
:10AC400010B504468068002809D0236801222046F8
:10AC50009847002803D0A068401EA060012010BDC6
:10AC600038B5002439B1012912D0022912D00529A2
:10AC70001DD0002038BD0546012269462846FFF751
:10AC8000B3FF90B19DF800000006F5D4012038BD57
:10AC900008220DE005466946FFF750FE28B1002165
:10ACA0002846009AFFF7A0FF38BD204638BD042291
:10ACB000BDE838400021FFF797BF000010B50C46F3
:10ACC000017A052908D0407A38B1084808A10268FD
:10ACD0002046FDF7B7FA00E01AB106A12046FDF7BD
:10ACE000B1FA2046BDE81040FDF7EABAC82B0020B3
:10ACF000257300000D0A00002DE9FC418046224822
:10AD000017460E46C5680A46012441462846FAF70A
:10AD10007FFB70B195F8550068B100F00101C0F3F8
:10AD2000400243462846CDE9006700F089F848B163
:10AD300009E0172407E03B4632464146284600F02A
:10AD400027F8F4E70524114D6FB1012C13D005F15C
:10AD50002400FBF749FE00BFFCF798FCC5F84880CB
:10AD60002046BDE8FC81012C02D0FCF78FFCF7E700
:10AD700001206861F4E7002231464046FAF71AF8EC
:10AD8000C5E90960E8E70000602B0020C04700200B
:10AD90002DE9F041044690F8550094B01D46174641
:10ADA000884620B1174940F22730F9F769F80126A3
:10ADB000CDE9007643460022214602A8F9F72EFE8F
:10ADC00000281CD0D5B1412202A90F48F7F72AFB71
:10ADD0000F4810490D4D401AC008042101EB0040F6
:10ADE0000DA1EE62FEF748F80020286294F8920068
:10ADF00010B194F8930008B96068A860012014B0FD
:10AE0000BDE8F081BCD10700614A0020C0470020A6
:10AE100068DB070038DB0700496E76616C696461A6
:10AE200074696E67206F6C64206170706C69636117
:10AE300074696F6E20696E2062616E6B20302E0027
:10AE40002DE9FF4FA5B0884604461546442113A8B6
:10AE5000329FF7F700FB442102A8F7F7FCFADDF870
:10AE6000A09058EA050004D13C4940F26130F9F75E
:10AE700007F83B483B4A801A02224FEAD00A02EB0D
:10AE80000A46B8F1000F1ED0A16D289800F01CFEF4
:10AE9000002848D02898FAF7D9FC4FF0010B20B1D0
:10AEA00030463149FDF7E8FFB5B3A16DCDE9001B90
:10AEB0000022214613A8289BF9F7B0FD002832D0C4
:10AEC000A06D81443F1A8DB10020CDE900704B4642
:10AED0004246214602A8F9F7A1FD002823D09DF89B
:10AEE000080018B130462149FDF7C6FF339898B3E2
:10AEF0001F4EB8F1000F1ED02898FAF7A7FC18B122
:10AF000006F11800FBF770FD412213A91948F7F765
:10AF100089FA5DB1AC200AE0FFE70BEB0A40164965
:10AF2000FDF7AAFF002029B0BDE8F08FA520F06250
:10AF3000A06D706301E0AA20F0626DB10D4841225E
:10AF400002A98230F7F76EFA94F8920010B194F8E3
:10AF5000930008B96068F0600120E4E7BCD1070005
:10AF600068DB070038DB070078D1070074D00700E2
:10AF7000C0470020204A0020C0CF070038B5C38852
:10AF80000D46044633B114A0009015A216A1284620
:10AF9000FDF758F9217A05291CD0607A48B1A088BC
:10AFA000FDF7CCFD164951F8202016A12846FDF7E3
:10AFB00049F9A0880021FEF709F803461049207AD4
:10AFC000143951F8202001B02846BDE830400EA1C8
:10AFD000FDF738B938BD00001B5B306D0000000084
:10AFE0001B5B313B33316D0025734C6F67732064FD
:10AFF000726F70706564202825642925730D0A001E
:10B00000C82B0020257300003C25733E2025733A91
:10B0100020000000EFF30580C005C00D01D0012025
:10B020007047EFF3148040F30000401C70470000AD
:10B03000034802490068FAF707BE0000882B002089
:10B0400024C707002DE9F041224C0025224E207A2A
:10B05000012730B92148311D0068FAF700FE306041
:10B0600038B1022020723168087928B101281CD13A
:10B0700014E06560BDE8F081D1E90503C01A142829
:10B0800000D31420B7EB900F01D2820800E0012218
:10B090000869C9681844194429DF03E0D1E90301AC
:10B0A000084428DF58B1112812D003213068FAF77C
:10B0B00064F925726560BDE8F041FFF7B9BF207CF7
:10B0C0000028D7D1BDE8F04100210220FDF724BBC4
:10B0D0002772CFE72C510020842B002024C70700C3
:10B0E00010B5074C201DFAF7D9FD002806D1607C69
:10B0F000002803D1BDE81040FFF7A4BF10BD000039
:10B100002C51002010B510461A46F7F78BF9002095
:10B1100010BD10B510461A46F7F784F9002010BD8F
:10B120002DE9F0411E681C461546074621B101294C
:10B1300018D0052923D119E000202060401C206090
:10B14000B0421CD8012229463846FFF74DFD0028A1
:10B1500006D015F8010B000601D52068EEE70120A6
:10B16000BDE8F08108200246186002E00420024693
:10B17000186029463846BDE8F041FFF735BD00208C
:10B18000EEE770B516460A460446C11C104600F0AC
:10B1900023FF054661193046C91C00F01DFF2844F5
:10B1A00070BD000003B5094A85B0D2E91612CDE999
:10B1B000001207498989ADF8001006A9CDE90210EF
:10B1C000044869464088AEDF07B000BD90C507005F
:10B1D000643000202C2B002008467047084670473A
:10B1E0002DE9F047FCF75EFBDFF8C480D8F830208B
:10B1F000D8F8347000EB020AB81A411EC1F30B01F3
:10B20000401A00F6FF792B492B48D8F84860081AF5
:10B21000C508042000EB0540044628A1FDF72CFEDC
:10B2200042F204002F4A8159012000EB054591426A
:10B2300006D028462CA1FDF71FFE0320BDE8F087AD
:10B24000D8F830000644B84205D1204633A1FDF7B6
:10B2500013FE0020F2E7C0B906F50050017814296A
:10B2600001D9416900E000213148B1FBF0F34FF40E
:10B2700040510A78142A01D9496900E00021B1FB44
:10B28000F0F220462BA1FDF702FE08234A46314684
:10B290005046FAF763F9040005D0284630A1FDF7BF
:10B2A000EBFD2046CAE7BDE8F0470020FCF7EABA0C
:10B2B000C047002088DB070038DB0700456E746557
:10B2C00072206E72665F626F6F746C6F616465721C
:10B2D0005F6466755F73645F636F6E74696E7565D6
:10B2E00000000000DBE5B151536F757263652061AA
:10B2F00064647265737320646F6573206E6F74206D
:10B30000636F6E7461696E20612076616C69642080
:10B31000536F66744465766963652E0053442061FB
:10B320006C726561647920636F7069656400000008
:10B3300040420F005570646174696E672053442E5B
:10B34000204F6C64205344207665723A2025642C8B
:10B35000204E6577207665723A2025640000000053
:10B360004661696C656420746F20636F7079206634
:10B3700069726D776172652E0000000070B50F482C
:10B380000F49401AC408042000EB04400DA1FDF74A
:10B3900073FDFFF725FF05004FF0010000EB0444AB
:10B3A00002D020460FA105E0F8F774FD050004D097
:10B3B000204612A1FDF760FD284670BD88DB07001E
:10B3C00038DB0700456E746572206E72665F6466D6
:10B3D000755F73645F626C5F636F6E74696E7565D1
:10B3E0000000000053442B424C3A20534420636F2A
:10B3F0007079206661696C656400000053442B42DB
:10B400004C3A20424C20636F7079206661696C650C
:10B4100064000000F0B50546002003464FF4405498
:10B420000C4E4FF6FE7712E0D4F804C0B44505D1B7
:10B4300055F823C0B4F80CE0F44504D02AB155F80F
:10B4400023C0BC4501D10120F0BD5B1CDBB28B42A7
:10B45000EAD3F0BDDBE5B15110B5040003D11A49C0
:10B460005320F8F70DFD4FF44050184940688842CA
:10B4700021D1218A71B1626904F11400002A94F883
:10B4800055200BD0042A07D00022BDE81040C9B2D5
:10B49000FFF7C0BF002010BD0122F6E712B1012A5C
:10B4A00007D1F7E7012904D9C9B20022FFF7B2FF9B
:10B4B000F0E7012010BD208A10B160690028E9D1B1
:10B4C00020780028F5D110BD04D20700DBE5B1518A
:10B4D0003EB504460B496846FEF75EF90AE0684649
:10B4E000FEF736F9D0E900212046904740B1684682
:10B4F000FEF790F96846FEF72BF90028EFD13EBD24
:10B5000011203EBDC8C907003EB504460A49684639
:10B51000FEF742F909E06846FEF71AF9D0E9002182
:10B52000204690476846FEF775F96846FEF710F921
:10B530000028F0D13EBD0000D4C907002DE9F0413C
:10B540001400884618D000250E4F032608EB05018D
:10B5500022460020F7F7D6FF0544241A40B9387870
:10B56000002809D008494FF47A408847761E05D054
:10B5700001203870002CE9D1BDE8F081002038703E
:10B58000FAE700008C2B0020A1C907002DE9F0414B
:10B590000E46074613481449144D401AC4080320A8
:10B5A00000EB044012A12A68FDF76AFC3046F9F767
:10B5B0001FFC20B919494FF4C170F8F761FC184B12
:10B5C0003A463146286800F053F8020007D00120BF
:10B5D00000EB0440BDE8F04112A1FDF751BCBDE80D
:10B5E000F081000058DB070038DB07005C2B0020EF
:10B5F0004261636B696E672075702073657474694E
:10B600006E6773207061676520746F206164647277
:10B6100065737320307825782E00000034CF070042
:10B6200040440020436F756C64206E6F7420706519
:10B6300072666F726D206261636B7570206F662039
:10B64000626F6F746C6F6164657220736574746986
:10B650006E677321204572726F723A2030782578B8
:10B660000000000000225821001DF9F7A3BB0000D4
:10B670002DE9F04715464FF460771E46894680460F
:10B680003A46F6F7FAFE224A224B0421D21AD20891
:10B6900001EB02440028204617D01FA1FDF7ECFB68
:10B6A0002046424621A1FDF7EBFB00220121404646
:10B6B000FBF700FC174A164B01219A1AD20801EB3E
:10B6C000024458B1204621A11DE02949FDF7D4FBD1
:10B6D0000DB10020A8470020BDE8F08726B9254914
:10B6E00040F25D10F8F7CCFB3A4649463046F6F793
:10B6F00099FE2B463A4631464046FBF791FC00281E
:10B70000EAD020461CA1FDF7B7FB0320E4E70000C8
:10B7100058DB070038DB070057726974696E6720D1
:10B7200073657474696E67732E2E2E004572617393
:10B73000696E67206F6C642073657474696E6773DB
:10B740002061743A2030782530387800436F756C6A
:10B7500064206E6F74206572617365207468652063
:10B7600073657474696E677320706167652100008A
:10B77000E8CE070034CF0700436F756C64206E6F0E
:10B78000742077726974652074686520444655207A
:10B7900073657474696E677320706167652100005A
:10B7A00070B516460D46040007D035B1206C8022D6
:10B7B00000213828225403D307E00E2070BD215405
:10B7C000401C3828FBD30BE02154401C4028FBD3FD
:10B7D0002146084600F096F838212046F6F73BFE51
:10B7E000216CD4E912304A0FC9003834591850413D
:10B7F000C4E90410227CE2710A0A42EA0062A271E2
:10B800000A0C42EA00426271020242EA11602071AF
:10B810006069E070010AA170010C6170000E04F80B
:10B8200038092146084600F06DF84FF00002EEB1ED
:10B83000E06ED100C840A854A36ECB40A818037195
:10B84000636ECB400372236ECB400373E36DCB403A
:10B850000374A36DCB400375636DCB400376236DFA
:10B86000CB40521C0377042AE2D31FE01823504236
:10B87000216D03EBC000C140A954666DC640A918F4
:10B880000E71A66DC6400E72E66DC6400E73266E32
:10B89000C6400E74666EC6400E75A66EC6400E7625
:10B8A000E66EC640521C0E77042AE0D3002070BD1D
:10B8B000A8B100210164C0E912110A4901650A49D1
:10B8C00041650A4981650A49C1650A4901660A4913
:10B8D00041660A4981660A49C166002070470E2008
:10B8E0007047000067E6096A85AE67BB72F36E3C7D
:10B8F0003AF54FA57F520E518C68059BABD9831F3B
:10B9000019CDE05B2DE9F04FC8B0002213466F4619
:10B91000CC181B1D2588A6786DBA2D04E47845EA5D
:10B920000625254347F82250521C102AF0D31BE06D
:10B9300007EB820151F8083C4FEA734484EAF34470
:10B9400084EA932451F83C3C4FEAF31585EAB34569
:10B9500085EAD303234451F81C4C51F8401C214480
:10B96000194447F82210521C402AE1D3036D479333
:10B97000416D4691846D4594C26D44929246026E2B
:10B980004392456E4295A946856E4195C66E409696
:10B99000B34600264FEAB21787EAF22787EA726CAD
:10B9A00002EA090725EA020887EA0807BC44204F93
:10B9B00057F8268008EB0B07BC445DF82670AB46B1
:10B9C0000CEB070E4FEAB30787EA733787EAB35CDD
:10B9D00081EA04074D4601EA040891461F400AEB3C
:10B9E0000E02A24687EA08070C46BC441946761C9C
:10B9F0000EEB0C03402ECDD3479E33440365469B8C
:10BA00001944416545992144816544995144C16572
:10BA10004399114401664299494441664199294438
:10BA2000816640995944C16648B0BDE8F08F000076
:10BA300090C807002DE9F04116460F46040004D0D7
:10BA400006B317B10025A8461AE00E20BDE8F08124
:10BA5000216C785D6054206C401C206440280ED11D
:10BA600021460846FFF74EFFD4E912014FF4007259
:10BA7000801841F10001C4F84080C4E912016D1C36
:10BA8000B542E5D30020E1E710B51620F7F7DEFE5A
:10BA900048B10C4882684FF4800152B1016821F42A
:10BAA0008001016010BDBDE8104042F20100F8F7CE
:10BAB00015B84FF0E020C0F88011BFF34F8FBFF3EF
:10BAC0006F8F10BD344F00202DE9F04100F500527A
:10BAD0001A481B4F0123C01B174CC008556803EBC5
:10BAE0000040A54201D017491FE04D1EC5F30B05CC
:10BAF000491B41F6FF75966829448E4201D21249CE
:10BB000013E04FF440514D68A54211D10C78102C30
:10BB100001D9096900E000211478102C01D91269BB
:10BB200000E00022914203D00849FDF7A5F9002367
:10BB30001846BDE8F0810000DBE5B15168DB070085
:10BB400038DB070024D10700B8D0070004D0070075
:10BB500010B51620F7F77AFEA0B1114890F800044E
:10BB60004009082811D20121814011F0EC0F0CD0BE
:10BB70000C4882684FF480016AB1016841F4800189
:10BB8000016010BD42F2010001E042F20200BDE896
:10BB90001040F7F7A3BF4FF0E020C0F8001110BD30
:10BBA00016E000E0344F00202DE9F0471E46924693
:10BBB00089460546040C089FF9F770FB8046FDF79F
:10BBC000FBF9A04204D80FA140F2A910F8F758F9E8
:10BBD00044EA0841741C1B483C4000EB84023E4090
:10BBE00000EB8600D160C16865F3C5016AF3891175
:10BBF00069F39F2121F00301491C21F00401C16078
:10BC0000BDE8F0872E2E5C2E2E5C2E2E5C2E2E5C38
:10BC10002E2E5C636F6D706F6E656E74735C6C69F5
:10BC2000627261726965735C6C6F675C7372635C8E
:10BC30006E72665F6C6F675F66726F6E74656E645E
:10BC40002E630000D85200202DE9FC47814617489A
:10BC50001746884605681C46012201A91846F9F7CF
:10BC600019F8134EB8B101998B1C00200AE000BFEF
:10BC700057F8202003EA050C06EB8C0C401C5B1CDB
:10BC8000CCF80C20A042F3D30B462246414648464E
:10BC90000095FFF789FF307802E000BFFCF77CFFDA
:10BCA0000028FBD1F9F753FEBDE8FC87982B002054
:10BCB000D85200202DE9FF41324800F15C01826B2F
:10BCC0006846FEF759FF304F9DE8070007F11C0357
:10BCD0002F4C83E8070019462C48C8600020A0704C
:10BCE0006060A0604FF44771A7F54070F6F7B3FBB2
:10BCF000A7F54072274902F54770FEF7A5FC2649D3
:10BD0000264A891AC908012202EB014578B1A078B8
:10BD100038B1A7F5407090F86C110029017826D051
:10BD200041B128461EA100BFFDF7A6F828E028462D
:10BD300023A1F9E790F8720110B3D4E901122C4E57
:10BD40006846FEF719FF9DE80F001C3787E80F00D3
:10BD50004FF4B2713046F6F77EFB3246254906F5C0
:10BD6000D470FEF771FC30B9284623A1DCE739B165
:10BD7000807928B12F4E0120E66004B0BDE8F08143
:10BD80000020FAE7C0470020404E002089A90700A4
:10BD9000602B002060C5070068DB070038DB070068
:10BDA00048616E646C65723A20496E76616C6964B4
:10BDB00020696E697420636F6D6D616E642E000082
:10BDC00048616E646C65723A20496E76616C696494
:10BDD0002070726F746F636F6C2062756666657237
:10BDE000206D5F70625F73747265616D00000000AA
:10BDF000B44C002040C4070048616E646C65723A20
:10BE000020496E76616C69642070726F746F636F25
:10BE10006C20627566666572206D5F70625F737418
:10BE20007265616D2028696E697420636F6D6D6144
:10BE30006E642900484B00202DE9F0410F4605466D
:10BE4000234824492A46401AC008042101EB004037
:10BE500021A1FDF715F8B7F1807F03D324498F2086
:10BE6000F8F70EF8962F03D221499020F8F708F83A
:10BE70006FF07F40874200D238461E4ED6F8041538
:10BE80000144381A21F07F44411E6860952902D28E
:10BE90009630963C68602D7B042D03D3144977209F
:10BEA000F7F7EEFF06EB8500C0F8404512494FF466
:10BEB000F86088474FF4A07000EB85013046FDF72D
:10BEC0001DFA4FF48030A840C6F80403BDE8F081A5
:10BED00088DB070038DB070074696D65725F61639A
:10BEE000746976617465202830782578290000000F
:10BEF00054CB070000400240B1C3070070B5174E95
:10BF00003078002829D1164800680125C0F3004088
:10BF100008B914480560144C4FF480712046FDF7B1
:10BF2000EDF94FF4A0712046FDF7E8F94FF4A27146
:10BF30002046FDF7E3F90D4A0020A02182F8001405
:10BF40000A4A1021203AC2F80011C4F80805A56079
:10BF500025600220C4F80403357070BDF42A002067
:10BF600018040040080000400040024024E000E0C7
:10BF700070B515460E460446FFF7C0FF3146204611
:10BF80002560BDE87040FFF757BF000010B50446BC
:10BF900009480A492246401AC008042101EB004022
:10BFA00007A1FCF76DFF217B4FF4803088400949E1
:10BFB000C1F8080310BD000088DB070038DB07006C
:10BFC00074696D65725F73746F702028307825789E
:10BFD00029000000004002400870020A4A70020C6A
:10BFE0008A70000EC87004207047000010B5024827
:10BFF000F9F74BFE002010BD802B002010B5142156
:10C000000448F6F728FA04480068F9F7F7FD00201D
:10C0100010BD00002C51002024C707002DE9F05F5F
:10C020008346DDE90A4A994690460D4608460127AF
:10C0300003E000BFB0FBF8F07F1C4045FAD2B945E1
:10C0400000D94F465FEACA7012D18CB15FEA8A709C
:10C0500002D5B9F1000F01D0202607E0302605E017
:10C0600031465846641EF8F76FFE0CB1A742F7D36D
:10C070005FF00106B9F1010F02D9A9F1010903E04E
:10C08000B5FBF6F0404502D306FB08F6F2E7DFF811
:10C090003C9000BFB5FBF6F000FB165519F80010F8
:10C0A0005846F8F751FEB6FBF8F6002EF2D15FEADB
:10C0B000CA7009D0002C07D0A74205D220215846CB
:10C0C000641EF8F741FEF5E7BDE8F09FE8C60700FB
:10C0D0002DE9F041084601241646254600212B464D
:10C0E0000A46FAF78BFC0C490C4A891ACF0830B182
:10C0F00005EB07400AA1FCF7BFFE042409E0FAF7AC
:10C1000063FC02463060042000EB07400BA1FCF703
:10C11000B7FE2046BDE8F08168DB070038DB07008A
:10C1200043616E27742066696E6420726F6F6D20A4
:10C13000666F72207570646174650000577269746F
:10C140006520616464726573732073657420746F15
:10C1500020307825303878002DE9F0411C4B1D4FF8
:10C160000F2600240125DB1B90F85520DB0805EB8A
:10C1700003450AB1042A03D190F86430012B06D09C
:10C18000D30707D090F85630012B02D002E0846E1E
:10C190000DE0846D92070AD590F85C20012A06D143
:10C1A000026E0D48C0F5FC239A4204D814443CB1F9
:10C1B00001260C6008E0284608A1FCF768FE04266A
:10C1C00028460EA1FCF758FE3046BDE8F08100007D
:10C1D00068DB070038DB070000200700424C2073B3
:10C1E000697A652028256429206F766572206C693C
:10C1F0006D6974202825642900000000496E697467
:10C20000207061636B657420646F6573206E6F745A
:10C2100020636F6E7461696E2076616C696420665C
:10C2200069726D776172652073697A65000000003C
:10C2300030B100680549884205D048F20250704785
:10C2400048F2015070470020704700006E52464887
:10C2500070B5FDF775FB002811D00020084A094B86
:10C26000094C0121166801FA00F52E4203D004EBB7
:10C270008005C5F80036401CC0B20728F2D370BD57
:10C28000080501403546526E000001400748084944
:10C2900010B5401AC008032101EB004005A1FCF7CE
:10C2A000EBFDBDE81040FFF7D3BF000038DB07000F
:10C2B00038DB0700496E7465726E616C20666565D7
:10C2C0006400000000207047002070472DE9FC4109
:10C2D00080461C4617460E460C48089DF9F7DEFCC2
:10C2E00010B11120BDE8FC81A20839463046FCF7A8
:10C2F000D5FF0648F9F7C9FC33463A4601214046C6
:10C30000CDE90045F9F71EF80020EBE7802B00206F
:10C310002DE9F84F114D884681461E46174669465D
:10C32000DDF828A02868F9F784FC040013D01C214C
:10C33000F6F791F800202071C4F80090C4E9048653
:10C34000C4E902A769462868F9F794FCFEF7C8FE1D
:10C350000020BDE8F88F0420FBE7000024C7070099
:10C3600084B7AC5DBA001CCDBE4928F7CBD9744464
:10C370005DA08494DB12A36DB24A17A13D05B938C4
:10C38000DBA4214542101BBFEB09B53367AB911409
:10C390006DF5F17DD69D178820DFCFEC866407C14F
:10C3A0000338FDD870470D0E0F100B0C1819000044
:10C3B0000338FDD870470000359907003B99070006
:10C3C0001199070020000000780000000000000024
:10C3D0004800280000204000C1270700000000009E
:10C3E000010001000000000001000000000000004A
:10C3F0000200050001000000220000000000000013
:10C40000000000000000000000000000000000002C
:10C410000100010000000000010000000000000019
:10C4200002000500010000004200000000000000C2
:10C4300000000000000000000000000000000000FC
:10C44000010011000400FCFF0400000000000000D7
:10C45000020011000400FCFF0400000000000000C6
:10C46000030021000400FCFF040010000000000095
:10C47000040011000100FFFF0100000000000000A7
:10C48000050011000200FEFF040000000000000093
:10C49000060011000400FCFF040000000000000082
:10C4A000070011000400FCFF040000000000000071
:10C4B000080017000200FEFF24000000E0C3070090
:10C4C000090010000100FFFF01000000DCC30700AD
:10C4D0000A0027000200FEFF4400030010C407000A
:10C4E000000000000000000000000000000000004C
:10C4F000010011000100FFFF01000000000000002A
:10C50000020017000200FEFF6401000040C40700A3
:10C51000000000000000000000000000000000001B
:10C52000010007000000000068010000F0C40700DF
:10C5300002000100000000000100000000000000F7
:10C5400003000500010000004200000000000000A0
:10C5500000000000000000000000000000000000DB
:10C56000010017000400FCFF68010000F0C4070090
:10C57000020017000400FCFFAC01000020C507000A
:10C5800000000000000000000000000000000000AB
:10C590000011030000111300020000000100000060
:10C5A0000338FDD870470C000C0000005802000052
:10C5B0000200000000000000020000000000000077
:10C5C00028300020090000000000000000000000EA
:10C5D0000100000000000000280000000000000032
:10C5E0000000000000010000000001000000000049
:10C5F000000000000000000000000000000000003B
:10C60000BD40070000000000000000000000000026
:10C610000200000000000100000000000000000017
:10C620000800000000000000BD400700D5A2070080
:10C6300000000000000000000400000000000000F6
:10C6400000000000000000000000000000000000EA
:10C6500000000000000000000000000000000000DA
:10C66000F4000000000000001800000000000000BE
:10C6700000000000000000000000000000000000BA
:10C6800000000000000000000000000000000000AA
:10C69000170000000000000050EADA308883B89FDD
:10C6A000604F15F30000C98E02000000000000007A
:10C6B0000000000000000000040000000000000076
:10C6C000000000000000000000000000000000006A
:10C6D0000001000000000000000000000000000059
:10C6E00000000000000000003031323334353637AE
:10C6F0003839414243444546001000000400000020
:10C70000010000000D570700EDBF070005B107004D
:10C71000CDC20700B1520700D9B10700C5C207005A
:10C720002D580700404F00200010000004000000BA
:10C730000100000019570700FDBF070013B10700F3
:10C7400011C30700F9520700DDB10700C9C2070095
:10C750003D580700556E6B6E6F776E206572726F75
:10C760007220636F64650000000000001CD60700A3
:10C7700001000000C8D4070002000000BCD207007E
:10C78000030000003CD507000400000090D507001E
:10C790000500000070D40700060000000CD407005C
:10C7A0000700000078D507000800000084D40700C7
:10C7B00009000000E8D407000A00000004D60700C2
:10C7C0000B000000A4D207000C0000009CD407005E
:10C7D0000D0000006CD607000E00000068D50700B1
:10C7E0000F000000A4D5070010000000D8D50700F6
:10C7F0001100000080D607001200000054D6070088
:10C8000013000000F0D507008000000024D40700CA
:10C810008100000060D307008200000020D30700E1
:10C820008300000000D30700840000003CD3070011
:10C830008500000048D407008600000050D507009E
:10C8400090000000ECD3070091000000E0D2070048
:10C8500092000000B0D4070000820000B8D50700A5
:10C860000182000004D507000282000020D50700E5
:10C87000008400007CD307000184000028D6070054
:10C8800002840000C4D3070003840000A0D3070083
:10C89000982F8A4291443771CFFBC0B5A5DBB5E92B
:10C8A0005BC25639F111F159A4823F92D55E1CAB9F
:10C8B00098AA07D8015B8312BE853124C37D0C552D
:10C8C000745DBE72FEB1DE80A706DC9B74F19BC175
:10C8D000C1699BE48647BEEFC69DC10FCCA10C2465
:10C8E0006F2CE92DAA84744ADCA9B05CDA88F97649
:10C8F00052513E986DC631A8C82703B0C77F59BFB3
:10C90000F30BE0C64791A7D55163CA0667292914DE
:10C91000850AB72738211B2EFC6D2C4D130D38537B
:10C9200054730A65BB0A6A762EC9C281852C72923D
:10C93000A1E8BFA24B661AA8708B4BC2A3516CC76B
:10C9400019E892D1240699D685350EF470A06A10A4
:10C9500016C1A419086C371E4C774827B5BCB034F3
:10C96000B30C1C394AAAD84E4FCA9C5BF36F2E6891
:10C97000EE828F746F63A5781478C8840802C78C20
:10C98000FAFFBE90EB6C50A4F7A3F9BEF27871C623
:10C99000618A07005F8A0700598A070000000000CB
:10C9A0000338FDD870470000405200207F0000008F
:10C9B000C0520020D8DB0700E0DB070000000000C9
:10C9C0000000000001000007B4C90700C4C9070047
:10C9D00008000000ECC90700FCC9070008000000BF
:10C9E000FCC907000CCA070008000000F8DB0700BC
:10C9F00000DC07000000000000000000E8DB07008A
:10CA0000F8DB07000000000000000000000000004C
:10CA1000000000000000000000000000D0DB070064
:10CA2000D8DB07000000000000000000E82A00201A
:10CA30000CCA07002CCA070008000000E0DB070052
:10CA4000E8DB070000000000000000003CCA07000F
:10CA50004CCA070008000000F1A5070099A50700CF
:10CA600041A50700B7A40700BDA4070075A40700EF
:10CA7000C3A4070001A507000000000000404040DB
:10CA800040404040404041414141414040404040A1
:10CA9000404040404040404040404040400502024D
:10CAA000020202020202020202020202022020200C
:10CAB0002020202020202002020202020202909068
:10CAC0009090909010101010101010101010101066
:10CAD00010101010101010100202020202028888BA
:10CAE00088888888080808080808080808080808C6
:10CAF00008080808080808080202020240000000AE
:10CB00007DCA07002E2E5C2E2E5C2E2E5C2E2E5CF7
:10CB10002E2E5C636F6D706F6E656E74735C6C69E6
:10CB2000627261726965735C626F6F746C6F61646D
:10CB300065725C6E72665F626F6F746C6F61646564
:10CB4000725F6170705F73746172745F66696E6149
:10CB50006C2E63002E2E5C2E2E5C2E2E5C2E2E5CF8
:10CB60002E2E5C636F6D706F6E656E74735C6C6996
:10CB7000627261726965735C626F6F746C6F61641D
:10CB800065725C6E72665F626F6F746C6F61646514
:10CB9000725F6466755F74696D6572732E63000001
:10CBA0002E2E5C2E2E5C2E2E5C2E2E5C2E2E5C638A
:10CBB0006F6D706F6E656E74735C6C6962726172BA
:10CBC0006965735C626F6F746C6F616465725C6ED3
:10CBD00072665F626F6F746C6F616465725F6677B7
:10CBE0005F61637469766174696F6E2E6300000023
:10CBF00043524320636F6D7075746174696F6E206A
:10CC00006661696C656420666F7220636F70696528
:10CC100064206170703A20737263206372633A20FB
:10CC20003078253038782C20726573206372633A2F
:10CC300020307825303878004120536F6674446581
:10CC40007669636520686173206A75737420626514
:10CC5000656E206163746976617465642E20497421
:10CC60002773206C696B656C79207468617420612E
:10CC70006E206170706C69636174696F6E20776992
:10CC80006C6C20636F6D6520696D6D65646961749E
:10CC9000656C7900526563656976656420424C4530
:10CCA0005F47415454535F4556545F45584348418C
:10CCB0004E47455F4D54555F52455155455354209D
:10CCC00028726571756573743A2025642C2072652D
:10CCD000706C793A202564292E0000002E2E5C2EDF
:10CCE0002E5C2E2E5C2E2E5C2E2E5C636F6D706F74
:10CCF0006E656E74735C6C69627261726965735C97
:10CD0000626F6F746C6F616465725C626C655F64A6
:10CD100066755C6E72665F6466755F626C652E63D5
:10CD2000000000006E72665F6673746F7261676503
:10CD30005F777269746528616464723D25702C2088
:10CD40007372633D25702C206C656E3D25642062F6
:10CD500079746573292C207175657565207573610B
:10CD600067653A20256400004372656174696E67E7
:10CD700020746865206F626A6563742077697468DF
:10CD80002073697A652030782530387820776F7580
:10CD90006C64206F766572666C6F77206669726D61
:10CDA000776172652073697A652E204F66667365B8
:10CDB000742069732030782530387820616E6420C3
:10CDC0006669726D776172652073697A652069732F
:10CDD000203078253038782E000000002E2E5C2E72
:10CDE0002E5C2E2E5C2E2E5C2E2E5C636F6D706F73
:10CDF0006E656E74735C6C69627261726965735C96
:10CE0000626F6F746C6F616465725C6466755C6E92
:10CE100072665F6466755F7265715F68616E646C8F
:10CE200065722E6300000000526573657474696E4C
:10CE30006720626F6F746C6F6164657220736574D4
:10CE400074696E67732073696E6365206E656974BB
:10CE5000686572207468652073657474696E6773A1
:10CE60002070616765206E6F722074686520626152
:10CE7000636B7570206172652076616C696420282F
:10CE8000435243206572726F72292E00526573748B
:10CE90006F72696E672073657474696E677320665C
:10CEA000726F6D206261636B75702073696E63656C
:10CEB000207468652073657474696E67732070618F
:10CEC000676520636F6E74656E7473206172652090
:10CED000696E76616C6964202843524320657272E2
:10CEE0006F72292E0000000044657374696E6174CE
:10CEF000696F6E2073657474696E67732061726503
:10CF0000206964656E746963616C20746F20736F4F
:10CF1000757263652C207772697465206E6F74205A
:10CF20006E65656465642E20536B697070696E6709
:10CF30002E0000002E2E5C2E2E5C2E2E5C2E2E5CE3
:10CF40002E2E5C636F6D706F6E656E74735C6C69B2
:10CF5000627261726965735C626F6F746C6F616439
:10CF600065725C6466755C6E72665F6466755F733D
:10CF7000657474696E67732E630000002E2E5C2E3C
:10CF80002E5C2E2E5C2E2E5C2E2E5C636F6D706FD1
:10CF90006E656E74735C6C69627261726965735CF4
:10CFA000626F6F746C6F616465725C6466755C6EF1
:10CFB00072665F6466755F7574696C732E630000DA
:10CFC0004D616A6F722053442075706461746520EE
:10CFD000627574206E6F20424C2E2041626F727415
:10CFE00020746F2061766F696420696E636170617F
:10CFF0006369746174696E672074686520424C2EA1
:10D0000000000000546865206E657720536F6674D9
:10D01000446576696365206973206F6620612064CA
:10D020006966666572656E742066616D696C7920EB
:10D030007468616E207468652070726573656E74C3
:10D0400020536F66744465766963652E20436F6D67
:10D050007061746962696C6974792063616E6E6F66
:10D06000742062652067756172616E746565642EF7
:10D0700000000000426F6F742076616C6964617417
:10D08000696F6E206F6620626F6F746C6F6164658C
:10D0900072206973206E6F7420737570706F727474
:10D0A000656420616E642077696C6C20626520691C
:10D0B000676E6F7265642E0054686520536F6674E6
:10D0C0004465766963652073697A6520696E2074AA
:10D0D000686520696E666F20737472756374206969
:10D0E0007320746F6F20736D616C6C20636F6D7053
:10D0F000617265642077697468207468652073695B
:10D100007A65207265706F7274656420696E207430
:10D11000686520696E697420636F6D6D616E642E41
:10D120000000000054686520536F6674446576699A
:10D13000636520646F6573206E6F7420636F6E7417
:10D1400061696E20746865206D61676963206E7522
:10D150006D626572206964656E74696679696E676F
:10D16000206974206173206120536F667444657672
:10D170006963652E00000000496E76616C69646128
:10D1800074696E6720617070206265636175736594
:10D1900020697420697320696E636F6D70617469B2
:10D1A000626C6520776974682074686520536F66C7
:10D1B000744465766963652E000000002E2E5C2E97
:10D1C0002E5C2E2E5C2E2E5C2E2E5C636F6D706F8F
:10D1D0006E656E74735C6C69627261726965735CB2
:10D1E000626F6F746C6F616465725C6466755C6EAF
:10D1F00072665F6466755F76616C69646174696F9D
:10D200006E2E63002E2E5C2E2E5C2E2E5C2E2E5C3F
:10D210002E2E5C636F6D706F6E656E74735C6C69DF
:10D22000627261726965735C626F6F746C6F616466
:10D2300065725C6466755C6E72665F6466755F7667
:10D2400065725F76616C69646174696F6E2E6300EC
:10D250002E2E5C2E2E5C2E2E5C2E2E5C2E2E5C63D3
:10D260006F6D706F6E656E74735C6C696272617203
:10D270006965735C6578706572696D656E74616C03
:10D280005F73656374696F6E5F766172735C6E72F3
:10D29000665F73656374696F6E5F697465722E6330
:10D2A000000000004E52465F4552524F525F494EB9
:10D2B00056414C49445F4441544100004E52465F40
:10D2C0004552524F525F534F465444455649434589
:10D2D0005F4E4F545F454E41424C454400000000B4
:10D2E0004E52465F4552524F525F46454154555249
:10D2F000455F4E4F545F454E41424C45440000004F
:10D300004E52465F4552524F525F4D555445585FFD
:10D31000554E4C4F434B5F4641494C45440000003D
:10D320004E52465F4552524F525F4D555445585FDD
:10D330004C4F434B5F4641494C4544004E52465F7B
:10D340004552524F525F4D555445585F434F4E44DE
:10D350005F494E49545F4641494C45440000000036
:10D360004E52465F4552524F525F4D555445585F9D
:10D37000494E49545F4641494C4544004E52465F30
:10D380004552524F525F424C455F495053505F5295
:10D39000585F504B545F5452554E434154454400DE
:10D3A0004E52465F4552524F525F424C455F495084
:10D3B00053505F504545525F52454A45435445449A
:10D3C000000000004E52465F4552524F525F424CA1
:10D3D000455F495053505F4C494E4B5F444953435E
:10D3E0004F4E4E4543544544000000004E52465FA8
:10D3F0004552524F525F4150495F4E4F545F494D25
:10D40000504C454D454E5445440000004E52465F39
:10D410004552524F525F4E4F545F535550504F52EA
:10D42000544544004E52465F4552524F525F4D4F55
:10D4300044554C455F4E4F545F494E495449414C09
:10D44000495A4544000000004E52465F4552524F33
:10D45000525F4D4F44554C455F414C5245414459F4
:10D460005F494E495449414C495A45440000000027
:10D470004E52465F4552524F525F4E4F545F464F99
:10D48000554E44004E52465F4552524F525F494EF0
:10D4900056414C49445F5354415445004E52465FF7
:10D4A0004552524F525F444154415F53495A4500DF
:10D4B0004E52465F4552524F525F494F5F50454E64
:10D4C00044494E47000000004E52465F4552524FBD
:10D4D000525F5356435F48414E444C45525F4D495D
:10D4E0005353494E470000004E52465F4552524F3B
:10D4F000525F494E56414C49445F4C454E47544853
:10D50000000000004E52465F4552524F525F445257
:10D51000565F5457495F4552525F414E41434B005D
:10D520004E52465F4552524F525F4452565F5457D7
:10D53000495F4552525F444E41434B004E52465F55
:10D540004552524F525F494E5445524E414C000095
:10D550004E52465F4552524F525F53544F524147CD
:10D56000455F46554C4C00004E52465F4552524F67
:10D57000525F4E554C4C00004E52465F4552524F42
:10D58000525F494E56414C49445F504152414D0013
:10D590004E52465F4552524F525F4E4F5F4D454D82
:10D5A000000000004E52465F4552524F525F464FB8
:10D5B0005242494444454E004E52465F4552524FF6
:10D5C000525F4452565F5457495F4552525F4F561F
:10D5D000455252554E0000004E52465F4552524F42
:10D5E000525F494E56414C49445F41444452000009
:10D5F0004E52465F4552524F525F5245534F55521D
:10D60000434553004E52465F4552524F525F494E7A
:10D6100056414C49445F464C414753004E52465F89
:10D6200053554343455353004E52465F4552524F64
:10D63000525F424C455F495053505F4348414E4E04
:10D64000454C5F414C52454144595F4558495354FC
:10D65000530000004E52465F4552524F525F434FB7
:10D660004E4E5F434F554E54000000004E52465FF1
:10D670004552524F525F54494D454F55540000009A
:10D680004E52465F4552524F525F42555359000029
:10D690002E2E5C2E2E5C2E2E5C2E2E5C2E2E5C638F
:10D6A0006F6D706F6E656E74735C6C6962726172BF
:10D6B0006965735C6C6F675C7372635C6E72665FE6
:10D6C0006C6F675F64656661756C745F6261636BE4
:10D6D000656E64732E6300007761726E696E670019
:10D6E00064656275670000001B5B313B33306D0081
:10D6F0001B5B306D000000001B5B313B33316D0064
:10D700001B5B313B33326D001B5B313B33336D00B0
:10D710001B5B313B33346D001B5B313B33356D009C
:10D720001B5B313B33366D001B5B313B33376D0088
:10D73000696E666F000000006572726F7200000013
:10D740002E2E5C2E2E5C2E2E5C2E2E5C2E2E5C63DE
:10D750006F6D706F6E656E74735C6C69627261720E
:10D760006965735C6578706572696D656E74616C0E
:10D770005F73656374696F6E5F766172735C6E72FE
:10D78000665F73656374696F6E5F697465722E6836
:10D790000000000073645F626C655F6366675F73BF
:10D7A000657428292072657475726E65642025730E
:10D7B000207768656E20617474656D7074696E673A
:10D7C00020746F2073657420424C455F4741545468
:10D7D000535F4346475F534552564943455F43486D
:10D7E000414E4745442E000073645F626C655F6381
:10D7F00066675F73657428292072657475726E653B
:10D8000064202573207768656E20617474656D707F
:10D8100074696E6720746F2073657420424C455F95
:10D82000434F4D4D4F4E5F4346475F56535F5555EF
:10D8300049442E0073645F626C655F6366675F7363
:10D84000657428292072657475726E65642025736D
:10D85000207768656E20617474656D7074696E6799
:10D8600020746F2073657420424C455F47415454C7
:10D87000535F4346475F415454525F5441425F53A4
:10D88000495A452E0000000073645F626C655F6357
:10D8900066675F73657428292072657475726E659A
:10D8A00064202573207768656E20617474656D70DF
:10D8B00074696E6720746F2073657420424C455FF5
:10D8C000434F4E4E5F4346475F4741502E00000096
:10D8D00073645F626C655F6366675F736574282954
:10D8E0002072657475726E65642025732077686593
:10D8F0006E20617474656D7074696E6720746F203A
:10D9000073657420424C455F4741505F4346475F13
:10D91000524F4C455F434F554E542E0073645F6227
:10D920006C655F6366675F73657428292072657430
:10D9300075726E6564202573207768656E2061744A
:10D9400074656D7074696E6720746F2073657420E0
:10D95000424C455F434F4E4E5F4346475F474154FD
:10D96000542E00006E72665F626F6F746C6F61643C
:10D9700065725F77647400006E72665F6466755FDF
:10D98000626C65006E72665F6466755F666C61737B
:10D99000680000006E72665F6466755F7265715F35
:10D9A00068616E646C6572006E72665F6466755F56
:10D9B00073657474696E6773000000006E72665F51
:10D9C0006466755F73657474696E67735F7376639D
:10D9D000690000006E72665F6466755F76616C69EF
:10D9E000646174696F6E00006E72665F6466755F75
:10D9F0007665725F76616C69646174696F6E000050
:10DA00006D656D5F6D6E6772000000006E72665F1F
:10DA10006673746F72616765000000007274745FF2
:10DA20006C6F675F6261636B656E6400617070004C
:10DA30006E72665F736468006E72665F7364685FBF
:10DA4000626C65006E72665F7364685F736F63001B
:10DA500008200001FFFFFFFFFFFFFFFFFFFFFFFFA9
:10DA600000000000000000000000000001000000B5
:10DA7000FFFFFFFF512563FCC2CAB9F3849E17A7BD
:10DA8000ADFAE6BCFFFFFFFFFFFFFFFF0000000055
:10DA9000FFFFFFFF96C298D84539A1F4A033EB2DC4
:10DAA000817D0377F240A463E5E6BCF847422CE1B0
:10DAB000F2D1176BF551BF376840B6CBCE5E316BF4
:10DAC0005733CE2B169E0F7C4AEBE78E9B7F1AFEB8
:10DAD000E242E34F4B60D2273E3CCE3BF6B053CC04
:10DAE000B0061D65BC86987655BDEBB3E7933AAAA0
:10DAF000D835C65A6F260700F933070015320700DC
:10DB00000CDC0700E82A0020200100002E38070066
:10DB10002CDD0700082C0020786700003E38070045
:10DB2000B9420700DD41070090C90700000000006E
:10DB30001CDA0700902B002064D9070000000404C1
:10DB400078D907000000040484D907000000040409
:10DB500094D9070000000404A8D9070000000404B9
:10DB6000BCD9070000000404D4D907000000040455
:10DB7000E8D907000000040400DA070000000000F4
:10DB80000CDA0700000004042CDA0700000004048B
:10DB900030DA07000000030338DA0700000003034F
:10DBA00044DA0700000003033C2B002078300020FB
:10DBB000893000208C300020F4000000A42B0020CD
:10DBC0009C2B0020A42B0020805100201800000076
:10DBD000AD43070000000000E186070000000000E0
:10DBE00019870700000000007D9507000000000075
:10DBF0000997070000000000F986070000000000F8
:10DC0000000000000300000039740700000000005D
:10DC1000000000000000000000000000042B0020B5
:10DC2000142B002000000000000000000000000095
:10DC300000000000000000000000000000000000E4
:10DC400000000000010000000000000000000000D3
:10DC5000FF00FFFF000000000000000000000000C7
:10DC600000000000000000000000000000000000B4
:10DC700001000000000000000000000000000000A3
:10DC800000E00700000000000000000000000000AD
:10DC90000000000000000000000000000000000084
:10DCA0000000000000000000000000000000000074
:10DCB0000000000000000000FF000000FF03000063
:10DCC0000000000000000000000000000000000054
:10DCD00000000000000000000000000038D707002E
:10DCE000D8D6070030D70700E0D60700F0D60700E7
:10DCF000E8D60700F8D6070000D7070008D70700C6
:10DD000010D7070018D7070020D7070028D707002B
:10DD1000000000000090D0030000000000000000A0
:0CDD2000D55007000010000000000800B3
:020000041000EA
:0410140000200700B1
:020000041000EA
:0410180000E00700ED
:0400000500072201CD
:00000001FF
